:020000040800F2
:1000000000160020450100084F1E0008471E00088A
:100010004B1E0008B3030008712200080000000016
:100020000000000000000000000000006522000841
:10003000B703000800000000511E000867220008F6
:100040005F0100085F0100085F0100085F01000810
:100050005F0100085F010008B9030008E70300081A
:10006000F1030008FB030008050400085F01000815
:100070005F0100085F0100085F0100085F010008E0
:100080005F0100085F0100085F0100085F010008D0
:100090005F0100085F0100085F0100080F0400080D
:1000A0005F0100085F0100085F0100085F010008B0
:1000B0005F0100085F0100085F0100085F010008A0
:1000C0005F0100085F0100085F0100087D1E000855
:1000D0008D1E00085F0100085F0100085F01000835
:1000E000C30300085F0100085F0100085F0100080A
:1000F0005F0100085F0100085F0100085F01000860
:100100005F0100085F0100085F0100089D1E0008F4
:100110005F0100085F0100085F0100085F0100083F
:100120005F0100085F0100085F0100085F0100082F
:10013000DFF80CD000F0CEF8004800478B5D0008D7
:10014000001600200648804706480047FEE7FEE705
:10015000FEE7FEE7FEE7FEE7FEE7FEE7FEE7FEE777
:100160006F22000831010008202A04DB203A21FA1E
:1001700002F00021704721FA02F3D040C2F12002C0
:10018000914008431946704700487047886B000843
:1001900040EA01039B0703D009E008C9121F08C009
:1001A000042AFAD203E011F8013B00F8013B521E89
:1001B000F9D27047D2B201E000F8012B491EFBD200
:1001C00070470022F6E710B513460A460446194662
:1001D000FFF7F0FF204610BD30B505462A460B4616
:1001E00012F8010B13F8014B08B1A042F8D01CB172
:1001F000002802D06D1CF1E7284630BDCAB2401E6F
:1002000010F8011F8A4202D00029F9D1002070475E
:10021000421C10F8011B0029FBD1801A704770B5F1
:10022000064603F081F9046805460A22002130469B
:1002300000F018F82C6070BD30B50B460146002068
:100240002022012409E021FA02F59D4205D303FA98
:1002500002F5491B04FA02F52844151EA2F1010219
:10026000F1DC30BD2DE9F04791460F46804604464B
:10027000002614F8015B2DB1FFF786FF0068405D92
:10028000C007F6D12B2D02D02D2D18D0641E4A4662
:100290003946204600F030F827B13968A14201D133
:1002A000C7F8008071054FF002040BD540420028CA
:1002B00003DD03F039F90460A007BDE8F08746F4D8
:1002C0008066E4E70028F8DA03F02EF904606FF0A6
:1002D0000040F2E7064C074D06E0E06840F00103FD
:1002E00094E8070098471034AC42F6D3FFF724FF98
:1002F0008C6B0008AC6B00082DE9F05F824600783B
:10030000002715468B460AF10104B946302801D072
:100310009DB113E014F8010B0127782803D0582869
:1003200001D045B10AE00DB1102D07D100271025ED
:1003300014F8010B02E0082500E00A250026B0466B
:100340000EE005FB080005FB06F1012701EB104656
:100350001FFA80F8B6F5803F00D3B94614F8010BB8
:10036000294600F018F80028EBDABBF1000F05D0A1
:100370000FB1641E00E05446CBF80040B9F1000F05
:1003800006D003F0D1F802210160C81EBDE8F09F3D
:1003900048EA0640FAE73A2800D2303820F0200236
:1003A000412A01D3A2F13700884201D34FF0FF3038
:1003B000704700BFFEE7704710B5012000F04AFB10
:1003C00010BD10B54FF4806000F044FB4FF40060A6
:1003D00000F040FB4FF4805000F03CFB4FF4005025
:1003E00000F038FB10BD10B5022000F033FB10BD4B
:1003F00010B5042000F02EFB10BD10B5082000F051
:1004000029FB10BD10B5102000F024FB10BD704773
:100410000021074AD1610749096941F00401054AF1
:1004200011611146096941F04001116170470000F6
:1004300048000020002002400021074AD1610749FE
:10044000096941F00201054A1161114648610969D3
:1004500041F0400111617047480000200020024037
:100460000022054BDA61054A126942F00102034B92
:100470001A610180704700004800002000200240FF
:1004800000201E49C96801F0100139B11C49C96931
:1004900041F002011A4AD16140F010001749C968C1
:1004A00001F0040139B11649C96941F00101144A4A
:1004B000D16140F004001149C96901F0010169B13D
:1004C0000F49C96941F004010D4AD16100BF0B49D0
:1004D000C96921F00101094AD16100BF00BF40F2A2
:1004E0000111884206D10549C96921F00101034A79
:1004F000D16101E00149C86000BF7047002002409F
:100500004800002070B5044600F058FC054609E09C
:10051000601C38B124B100F051FC401BA04201D94D
:10052000032070BD1248C06800F001000028EFD120
:100530000F48C06800F0200020B100BF20200C4907
:10054000C86000BF0A48C06800F0100048B90848F9
:10055000C06900F0010020B90548C06800F004003F
:1005600018B1FFF78DFF0120DBE70020D9E700007D
:100570000020024070B50446002594F821000228AE
:1005800003D00420A0630125C1E02068006820F0AA
:100590000E00216808602068006820F001002168D2
:1005A00008605C492068884252D95A4978392068E5
:1005B000884201D1012047E05649643920688842C9
:1005C00001D1102040E0534950392068884201D1C0
:1005D000801539E04F493C392068884201D18014A8
:1005E00032E04C4928392068884202D14FF48030EB
:1005F0002AE0484914392068884202D14FF480101B
:1006000022E044492068884201D140041CE042496C
:100610002068884201D1012016E03F49143120684A
:10062000884201D110200FE03B49283120688842E0
:1006300001D1801508E038493C312068884201D159
:10064000801401E04FF480303349091F086051E005
:10065000304978392068884201D1012047E02D498E
:1006600064392068884201D1102040E0294950397E
:100670002068884201D1801539E026493C3920683C
:10068000884201D1801432E022492839206888420A
:1006900002D14FF480302AE01E4914392068884284
:1006A00002D14FF4801022E01A492068884201D11B
:1006B00040041CE018492068884201D1012016E05E
:1006C000154914312068884201D110200FE01249E9
:1006D00028312068884201D1801508E00E493C315C
:1006E0002068884201D1801401E04FF4803009492C
:1006F00080394860012084F8210000BF002084F880
:10070000200000BF606B10B12046616B884728460F
:1007100070BD000080000240080402402DE9F04155
:1007200004460E460127002500BF2648007E01280A
:1007300002D10220BDE8F08101202249087600BFE5
:100740002068022813D14CF25030FFF7DBFE90BB3B
:100750000120FFF75DFE4CF25030FFF7D3FE074655
:100760001948006920F004001749086123E04CF2A1
:100770005030FFF7C7FEF0B94FF0FF303060A5688A
:1007800012E02846FFF758FE4CF25030FFF7BAFE51
:1007900007460D48006920F002000B4908610FB1BF
:1007A000356007E005F50065D4E9021001EBC020D3
:1007B000A842E6D800BF00BF00200249087600BF6B
:1007C0003846B7E74800002000200240034800698F
:1007D00040F080000149086100207047002002407D
:1007E0002DE9FE4F05468B46174698460126002404
:1007F0000020029000BF2448007E012802D1022080
:10080000BDE8FE8F01202049087600BF4CF2503031
:10081000FFF778FE064686BB012D02D1012002902B
:1008200006E0022D02D10220029001E00420029095
:1008300000241EE02201B946C24648465146FFF751
:1008400093FC80B20190022000FB04B0009001995B
:10085000FFF706FE4CF25030FFF754FE06460B48F9
:10086000006920F001000949086106B104E0601C3C
:10087000C4B202988442DDDB00BF00BF0020024901
:10088000087600BF3046BBE7480000200020024049
:1008900000200849096901F0800151B10649054A63
:1008A0005160064951601146096901F0800101B1AA
:1008B000012070470020024023016745AB89EFCD3E
:1008C0002DE9F04102460B4600208BE001278740CE
:1008D00007EA030100297DD0464F4FEA900C57F8F4
:1008E0002C4087074FEA177C0F2707FA0CF73C408C
:1008F000414FBA4201D1002719E0404FBA4201D11D
:10090000012714E03E4FBA4201D102270FE03D4FCC
:10091000BA4201D103270AE03B4FBA4201D1042772
:1009200005E03A4FBA4201D1052700E006274FEA19
:10093000807C4FEA1C7C07FA0CF7A74230D187076E
:100940004FEA177C0F2707FA0CF42A4F4FEA900C56
:1009500057F82C70A743DFF89CC04FEA90084CF87A
:1009600028702B4F3F688F43DFF8A4C0CCF800708D
:100970000CF104073F688F430CF1040CCCF80070B5
:100980000CF104073F688F430CF1040CCCF80070A5
:100990000CF104073F688F430CF1040CCCF8007095
:1009A000FF2901D8174600E0171D3D46FF2901D851
:1009B000870002E0A0F10807BF003E462F684FF015
:1009C0000F0C0CFA06FC27EA0C074FF0040C0CFA8B
:1009D00006FC00E005E047EA0C072F60D7688F436C
:1009E000D760401C23FA00F7002F7FF46FAFBDE8FB
:1009F000F08100000800014000080140000C0140A7
:100A0000001001400014014000180140001C01408A
:100A10000004014010B50446B4F5806F0ED0B4F563
:100A2000006F0BD0B4F5805F08D0B4F5005F05D03F
:100A3000B4F5804F02D0B4F5004F07D1044890F8C8
:100A40003000012802D10249486B804710BD0000E8
:100A50007001002010B5044604480068204020B111
:100A6000024804602046FFF7D5FF10BD1404014082
:100A70002DE9F847024600239C467BE14FF0010830
:100A800008FA03F4D1F8008008EA0400A0427DD1FE
:100A9000DFF8F4A2D1F80480A8EB0A09D0453AD0D7
:100AA00014DCB8F1030F50D009DCB8F1000F31D0DD
:100AB000B8F1010F1CD0B8F1020F49D120E0B8F114
:100AC000110F18D0B8F1120F42D11EE0B9F5881FEE
:100AD00025D006DCB9F5803F20D0B9F5801F37D18D
:100AE0001AE0B9F5001F18D0B9F5041F30D117E08E
:100AF000D1F80CC02DE0D1F80C8008F1040C28E0EE
:100B0000D1F80C8008F1080C23E0D1F80C8008F132
:100B10000C0C1EE000BF00BF00BF00BF00BF00BF45
:100B2000D1F80880B8F1000F02D14FF0040C0BE0AF
:100B3000D1F80880B8F1010F03D14FF0080C14610F
:100B400002E04FF0080C546103E04FF0000C00E0AD
:100B500000BF00BFFF2801D8904601E002F1040861
:100B60004646FF2802D84FEA830803E0A3F10808AD
:100B70004FEA88084746D6F800804FF00F0909FA77
:100B800007F928EA09080CFA07F900E07AE048EAD0
:100B90000908C6F80080D1F8048008F08058B8F140
:100BA000805F6FD100BFDFF8E481D8F8188048F08B
:100BB0000108DFF8D891C9F81880C846D8F818801D
:100BC00008F00108CDF8008000BF00BF4FEAB93837
:100BD0004FEA930958F829504FEA83784FEA187979
:100BE0004FF00F0808FA09F825EA0805DFF8A08198
:100BF000424502D14FF0000824E0DFF898814245D9
:100C000002D14FF001081DE0DFF88C81424502D18E
:100C10004FF0020816E0DFF88481424502D14FF020
:100C200003080FE0DFF87881424502D14FF0040855
:100C300008E0DFF87081424502D14FF0050801E07D
:100C40004FF006084FEA83794FEA197908FA09F854
:100C500048EA0505DFF850814FEA930948F8295022
:100C6000D1F8048008F48038B8F5803F0BD1DFF864
:100C70003C81D8F8008048EA0008DFF83091C9F8D4
:100C800000800AE075E0DFF82481D8F8008028EAC7
:100C90000008DFF81891C9F80080D1F8048008F442
:100CA0000038B8F5003F0ED1DFF8008108F10408E4
:100CB000D8F8008048EA0008DFF8F09009F104094C
:100CC000C9F800800DE0DFF8E48008F10408D8F8E6
:100CD000008028EA0008DFF8D49009F10409C9F877
:100CE0000080D1F8048008F48018B8F5801F0ED178
:100CF000DFF8B88008F10808D8F8008048EA000852
:100D0000DFF8A89009F10809C9F800800DE0DFF8C4
:100D10009C8008F10808D8F8008028EA0008DFF86D
:100D20008C9009F10809C9F80080D1F8048008F412
:100D30000018B8F5001F0ED1DFF8708008F10C081C
:100D4000D8F8008048EA0008DFF8609009F10C0943
:100D5000C9F800800DE0DFF8548008F10C08D8F8DD
:100D6000008028EA0008DFF8449009F10C09C9F86E
:100D700000805B1CD1F8008028FA03F8B8F1000F5E
:100D80007FF47CAEBDE8F88700001110001002402F
:100D900000080140000C0140001001400014014017
:100DA00000180140001C01400800014000040140FF
:100DB0000AB1016101E00B0403617047014800685A
:100DC00070470000040000200348006803490978C8
:100DD0000844014908607047040000200C0000200E
:100DE00010B50848006840F010000649086003206C
:100DF00000F0A2F80F2000F007F800F02BF8002018
:100E000010BD00000020024070B504460E48007876
:100E10004FF47A71B1FBF0F00C490968B1FBF0F5C1
:100E2000284600F0F6FF08B1012070BD102C07D253
:100E300000222146501E00F041F80548046001E000
:100E40000120F2E70020F0E70C0000200000002065
:100E5000080000207047000010B501460846002831
:100E600017DB00F01F0301229A400B4B440943F8A3
:100E7000242000BF00BF00BFBFF34F8F00BF00BFE3
:100E800000BF00BF00BF00BFBFF36F8F00BF00BF38
:100E900000BF00BF10BD000080E100E00146084631
:100EA000002809DB00F01F0301229A4043099B0040
:100EB00003F1E023C3F8002100BF70472DE9F05F84
:100EC00080460D461646002702F012FB07463946BB
:100ED0002A46334601F00700C0F1070ABAF1040FB1
:100EE00002D94FF0040A01E0C0F1070AD14600F12F
:100EF000040ABAF1070F02D24FF0000A01E0A0F194
:100F0000030AD4464FF0010A0AFA09FAAAF1010AC3
:100F10000AEA020A0AFA0CFA4FF0010B0BFA0CFB70
:100F2000ABF1010B0BEA030B4AEA0B0421464046E6
:100F300002F0E6FABDE8F09F00BF00F00702064BA2
:100F400019684FF6FF031940044B0B4343EA022193
:100F5000014B196000BF70470CED00E00000FA057E
:100F600070B504460D460CB9012070BD5A480068A2
:100F700000F00700A8420ED25748006820F0070092
:100F80002843554908600846006800F00700A84259
:100F900001D00120E9E7207800F0020002281DD1ED
:100FA000207800F00400042805D14C48406840F443
:100FB000E0604A494860207800F00800082805D120
:100FC0004648406840F4605044494860434840689F
:100FD00020F0F000A168084340494860207800F004
:100FE000010078B36068012806D13C48006800F42D
:100FF000003090B90120B8E76068022806D1374870
:10100000006800F0007040B90120AEE73348006886
:1010100000F0020008B90120A7E73048406820F03E
:101020000300616808432D494860FFF7C7FE064684
:1010300009E0FFF7C3FE801B41F28831884202D9E4
:10104000032092E707E02548406800F00C00616843
:10105000B0EB810FEDD12048006800F00700A842F6
:101060000ED91D48006820F0070028431A4908607F
:101070000846006800F00700A84201D0012074E78C
:10108000207800F00400042807D11448406820F4B8
:10109000E060E168084311494860207800F00800EA
:1010A000082808D10D48406820F46050216940EAC2
:1010B000C1000A49486000F0A1F808494968C1F335
:1010C0000311074A515CC840064908600648006899
:1010D000FFF79AFE002048E700200240001002407F
:1010E00076660008000000200800002010B5FFF719
:1010F00065FE04463D48006840F001003B49086039
:1011000006E0FFF75BFE001B022801D9032010BD9B
:101110003648006800F002000028F2D0334800682A
:1011200020F0F80040F0800030490860FFF746FEEC
:10113000044600202D49486008E0FFF73FFE001BF1
:1011400041F28831884201D90320E0E7274840680E
:1011500000F00C000028F0D12548264908602648F8
:101160000068FFF751FE08B10120D0E7FFF726FE27
:1011700004461E48006820F080701C49086006E0A4
:10118000FFF71CFE001B022801D90320BFE7174808
:10119000006800F000700028F2D114494860FFF7A1
:1011A0000DFE04461148006820F410200F49086025
:1011B00006E0FFF703FE001B642801D90320A6E721
:1011C0000A48006800F400300028F2D1074800689F
:1011D00020F48020054908600846406A40F080708D
:1011E00048620020886000BF91E7000000100240C4
:1011F00000127A000000002008000020F0B585B041
:101200000FF26C0C9CE8E01001A8A0E8E0101CA50F
:101210002D68009500210022002300240020194D94
:10122000696801F00C05F5B1042D02D0082D19D123
:1012300001E0154819E001ADC1F38346AC5D01F44E
:10124000803555B10F4D6D68C5F340451DF805203B
:101250000D4D6543B5FBF2F302E00C4D04FB05F3C5
:10126000184602E000BF084800BF00BF05B0F0BD4F
:1012700002030405060708090A0B0C0D0E0F1010D7
:10128000010200000010024000127A0000093D0037
:10129000F8B504460CB90120F8BD207800F0010033
:1012A000002878D0F848406800F00C0004280CD0E2
:1012B000F548406800F00C00082811D1F248406859
:1012C00000F48030B0F5803F0AD1EF48006800F4A8
:1012D000003000285FD0606800285CD10120DBE787
:1012E00000BF6068B0F5803F06D1E748006840F471
:1012F0008030E549086028E0606858B9E248006835
:1013000020F48030E04908600846006820F480201E
:1013100008601AE06068B0F5A02F0BD1DA480068C9
:1013200040F48020D84908600846006840F48030C6
:1013300008600AE0D448006820F48030D249086090
:101340000846006820F48020086000BF606888B10B
:10135000FFF734FD054606E0FFF730FD401B64282B
:1013600001D9032098E7C848006800F4003000283D
:10137000F2D010E0FFF722FD054606E0FFF71EFD64
:10138000401B642801D9032086E7BF48006800F4A9
:1013900000300028F2D1207800F00200022857D156
:1013A000B948406800F00C0050B1B748406800F000
:1013B0000C00082818D1B448406800F4803098B96F
:1013C000B148006800F0020020B12069012801D076
:1013D000012061E7AC48006820F0F800616940EA4C
:1013E000C100A949086033E02069E8B10120A7499C
:1013F0000860FFF7E3FC054606E0FFF7DFFC401B53
:10140000022801D9032047E79F48006800F0020046
:101410000028F2D09C48006820F0F800616940EA9A
:10142000C1009949086013E0002098490860FFF75F
:10143000C5FC054606E0FFF7C1FC401B022801D9A8
:10144000032029E79048006800F002000028F2D14C
:10145000207800F0080008282DD1A069B8B101203B
:101460008B490860FFF7AAFC054606E0FFF7A6FCDB
:10147000401B022801D903200EE78348406A00F090
:1014800002000028F2D0012000F0E4FC13E000206C
:101490007F490860FFF792FC054606E0FFF78EFCE7
:1014A000401B022801D90320F6E67748406A00F085
:1014B00002000028F2D1207800F00400042873D143
:1014C00000277148C06900F0805070B900BF6E48B5
:1014D000C06940F080506C49C8610846C06900F09E
:1014E0008050009000BF00BF01276A48006800F4E8
:1014F0008070B0B96748006840F480706549086042
:10150000FFF75CFC054606E0FFF758FC401B64282B
:1015100001D90320C0E65F48006800F4807000280D
:10152000F2D000BFE068012806D15748006A40F0B9
:1015300001005549086227E0E06858B95248006A3E
:1015400020F00100504908620846006A20F00400BB
:10155000086219E0E06805280BD14B48006A40F0AA
:101560000400494908620846006A40F00100086228
:101570000AE04548006A20F0010043490862084635
:10158000006A20F00400086200BFE068A0B1FFF725
:1015900015FC054609E0FFF711FC401B41F28831BC
:1015A000884202D9032077E622E03748006A00F03B
:1015B00002000028EFD012E0FFF700FC054608E02B
:1015C000FFF7FCFB401B41F28831884201D9032020
:1015D00062E62D48006A00F002000028F0D1012FD9
:1015E00005D12948C06920F080502749C86100BF53
:1015F000E069C8B32448406800F00C00082860D0B7
:10160000E069022848D1002020490866FFF7D6FB90
:10161000054606E0FFF7D2FB401B022801D9032054
:101620003AE61948006800F000700028F2D1206AFC
:10163000B0F5803F07D11448406820F40030A1681D
:10164000084311494860D4E9080108430E49496834
:1016500021F4741108430C49486001200B490866C5
:10166000FFF7ACFB054607E03DE0FFF7A7FB401B9B
:10167000022801D903200FE60348006800F000703B
:101680000028F2D02FE0000000100240000042428B
:101690008004424200700040002014490866FFF7B1
:1016A0008DFB054606E0FFF789FB401B022801D9A8
:1016B0000320F1E50E48006800F000700028F2D128
:1016C00011E0E069012800D1E6E50948466806F422
:1016D0008031206A814204D106F47011606A81422F
:1016E00001D00120D8E50020D6E5000000004242EC
:1016F0000010024010B504460CB9012010BD0220B4
:1017000084F851002068006820F0400021680860DB
:10171000204600F00FF90020606584F8510000BFFA
:1017200084F8500000BF00BFE8E77047F8B50446F2
:101730002068466820688568C5F3801048B905F0C0
:10174000010030B1C6F3801018B12046216C8847E3
:10175000F8BDC5F3400030B1C6F3C01018B1204643
:10176000616C8847F4E7C5F3401018B9C5F38010E1
:10177000002871D0C6F3401000286DD0C5F380104A
:10178000F0B194F8510003280ED0606D40F00400D1
:10179000606500BF002000902068C068009020684D
:1017A0008068009000BF0BE000BF00200090206820
:1017B000C068009020688068009000BF00BFC7E745
:1017C000C5F3401088B1606D40F00100606500BF56
:1017D000002000902068806800902068006820F059
:1017E00040002168086000BF00BF606D70B32068D2
:1017F000406820F0E00021684860012084F8510032
:1018000006F0020010B906F0010000B3206840683D
:1018100020F0030021684860E06C50B10F48E16C93
:101820004863E06CFEF7A6FE18B1606D40F0400022
:101830006065A06C50B10948A16C4863A06CFEF7CC
:1018400099FE18B1606D40F04000606502E02046EE
:10185000FFF76BFF7CE7FFE700BF79E7492100084E
:1018600010B504460CB9012010BD606A38B9606833
:10187000B0F5827F00D105E00021E16102E00021A6
:1018800021616161A06AB0F5005F00D100BF94F8EA
:10189000510028B9002084F85000204600F0CAF812
:1018A000022084F851002068006820F04000216880
:1018B0000860A08800F48270218901F40441084383
:1018C000A18901F400610843217C01F00201084371
:1018D000217D01F001010843218B01F400710843CF
:1018E000217F01F0380108432021095D01F08001CA
:1018F0000843218D01F40051084321680860042148
:10190000A06901EA104021684860A06AB0F5005F54
:1019100003D1A08D80B2216808612068C06920F4DD
:1019200000602168C86100206065012084F85100D2
:10193000002099E710B504463449206888421DD13B
:101940003348806920F48050314988612021314832
:10195000FEF7B6FF20212F48FEF7B2FF80212D4869
:10196000FEF7AEFF4FF400612B48FEF7A9FF2320DE
:10197000FFF772FA00202949087045E028492068DD
:10198000884220D12248C06920F480402049C861A3
:101990004FF400512348FEF793FF4FF48041214854
:1019A000FEF78EFF4FF400411E48FEF789FF4FF40B
:1019B00080511C48FEF784FF2420FFF74DFA0020D9
:1019C0001949087020E01949206888421CD1104844
:1019D000C06920F400400E49C86108211148FEF793
:1019E0006FFF10210F48FEF76BFF20210D48FEF717
:1019F00067FF4FF400410748FEF762FF3320FFF70F
:101A00002BFA00200A49087010BD00000030014088
:101A10000010024000080140002001400D0000209D
:101A200000380040000C01400E000020003C004047
:101A30000F00002010B586B00446B14920688842E6
:101A400070D100BFAF48806940F48050AD498861D3
:101A50000846806900F48050019000BF00BF00BFBD
:101A60000846806940F0040088610846806900F0FB
:101A70000400019000BF00BF00BF0846806940F02D
:101A8000040088610846806900F00400019000BFEE
:101A900000BF00BF0846806940F004008861084626
:101AA000806900F00400019000BF00BF00BF08463D
:101AB000806940F4807088610846806900F4807015
:101AC000019000BF00BF202002900220039001205F
:101AD00004900320059002A98B48FEF7C9FF20203F
:101AE00002900120049002A98748FEF7C1FF8020E0
:101AF00002900120049002A98348FEF7B9FF4FF439
:101B0000006002900120049002A98048FEF7B0FF17
:101B1000002201212320FFF7D1F92320FFF7BEF98E
:101B2000ECE0FFE77A492068884273D100BF75482E
:101B3000C06940F480407349C8610846C06900F438
:101B40008040019000BF00BF00BF0846806940F0A0
:101B5000080088610846806900F00800019000BF15
:101B600000BF00BF0846806940F008008861084651
:101B7000806900F00800019000BF00BF00BF084668
:101B8000806940F0080088610846806900F008001C
:101B9000019000BF00BF00BF0846806940F0080008
:101BA00088610846806900F00800019000BF00BF0E
:101BB0004FF4005002900220039001200490032073
:101BC000059002A95348FEF753FF4FF4804002905E
:101BD0000120049002A94F48FEF74AFF4FF400404D
:101BE00002900120049002A94A48FEF741FF4FF4F9
:101BF000805002900120049002A94648FEF738FF69
:101C0000002201212420FFF759F92420FFF746F98B
:101C100074E0FFE74049206888426FD100BF39482F
:101C2000C06940F400403749C8610846C06900F403
:101C30000040019000BF00BF00BF0846806940F02F
:101C4000080088610846806900F00800019000BF24
:101C500000BF00BF0846806940F008008861084660
:101C6000806900F00800019000BF00BF00BF084677
:101C7000806940F0080088610846806900F008002B
:101C8000019000BF00BF00BF0846806940F004001B
:101C900088610846806900F00400019000BF00BF21
:101CA0000820029002200390002004900320059059
:101CB00002A91848FEF7DCFE1020029001200490D3
:101CC00002A91448FEF7D4FE2020029001200490BF
:101CD00002A91048FEF7CCFE4FF40040029001200C
:101CE0000390049002A90848FEF7C2FE00220121D9
:101CF0003320FFF7E3F83320FFF7D0F806B010BD2C
:101D00000030014000100240000801400020014066
:101D100000380040000C0140003C004070470000CB
:101D2000F0B50446002700BF94F85000012801D107
:101D30000220F0BD012084F8500000BF94F85150FB
:101D40006668012D08D0B6F5827F03D1A06808B976
:101D5000042D01D002274BE009B102B10BB90127D4
:101D600046E094F85100042802D0052084F8510080
:101D7000002060652163A386E386A263A387E387CF
:101D8000E06820B11E4820641E48606403E01E48DD
:101D900020641E486064A06AB0F5005F11D100BFE6
:101DA0002068006820F40050D4F800C0CCF800008F
:101DB0002068006840F40050D4F800C0CCF800005F
:101DC00000BF2068406840F0E000D4F800C0CCF8C4
:101DD00004002068006800F04000402807D0206818
:101DE000006840F04000D4F800C0CCF8000000BF0C
:101DF00000BF002084F8500000BF384699E700007B
:101E0000AD1E00088F1F0008191F0008E71F0008FB
:101E1000704770B504462546681EB0F1807F01D337
:101E200001200FE0681E4FF0E02148610F214FF0C4
:101E3000FF3001F065FB00204FF0E02188610720B2
:101E40000861002070BD00BFFEE700BFFEE77047DD
:101E50007047000008B508490968C9084FF47A724C
:101E6000B1FBF2F14143009100BF00BF00994A1E4F
:101E700000920029F9D108BD0000002010B50248E9
:101E8000FFF754FC10BD00006800002010B50248A8
:101E9000FFF74CFC10BD0000C000002010B5024848
:101EA000FFF744FC10BD00001801002010B50446E7
:101EB0002068C068A16B0880A06B801CA063E08FC5
:101EC000401EE087E08F88B9A06AB0F5005F02D1BC
:101ED0000748206410BD2068406820F04000216859
:101EE0004860E08E10B9204600F0AAF800BFF1E784
:101EF000F51E000838B50446002000902068C06830
:101F0000009000BF2068406820F0400021684860D1
:101F1000204600F095F838BD10B504462068007BD7
:101F2000A16B0870A06B401CA063E08F401EE0878F
:101F3000E08F88B9A06AB0F5005F02D1074820643D
:101F400010BD2068406820F0600021684860E08E85
:101F500010B9204600F074F800BFF1E7611F0008D7
:101F600038B5044600200090206800F10C05287860
:101F700000909DF800002068406820F06000216813
:101F80004860E08E10B9204600F05AF838BD10B510
:101F90000446206B00882168C860206B801C206389
:101FA000E08E401EE086E08ED8B9A06AB0F5005FF2
:101FB0000CD12068006840F48050216808602068D7
:101FC000406820F080002168486010BD20684068AB
:101FD00020F0800021684860E08F10B9204600F0B2
:101FE0002FF800BFF1E710B50446206B0078216898
:101FF0000873206B401C2063E08E401EE086E08E5C
:10200000D8B9A06AB0F5005F0CD12068006840F430
:102010008050216808602068406820F080002168B6
:10202000486010BD2068406820F08000216848604A
:10203000E08F10B9204600F003F800BFF1E7000080
:102040007CB504463F4800681821B0FBF1F04FF41E
:102050007A71B0FBF1F0642148430190FEF7AEFEC7
:1020600005462068406820F020002168486000BFD5
:10207000019820B9606D40F02000606508E001988B
:10208000401E01902068806800F002000028EFD018
:1020900000BF2A466421204600F060F818B1606D48
:1020A00040F020006065A06850B900BF002000909B
:1020B0002068C068009020688068009000BF00BF62
:1020C00020688068C0F3001008B3204600F05AF87A
:1020D000012817D184F85100606D40F0020060655E
:1020E00000BF2068006820F4005021680860206864
:1020F000006840F400502168086000BF2046FFF7E8
:1021000014FB1EE04FF6EF702168886019E0606DE7
:1021100088B994F85100042806D1012084F85100B0
:102120002046FFF7FBFD0CE0012084F8510020461B
:10213000FFF76EFE05E0012084F851002046FFF70E
:10214000F4FA7CBD0000002070B505466C6A0020E2
:10215000E087E0862046FFF7E8FA70BDF8B5044650
:102160000D4616462B46002280212046009600F0A0
:102170000DF828B1606D40F0200060650320F8BDC7
:102180000020FCE701460120704700002DE9F84FD0
:1021900004460D4690461E46DDF82890FEF70EFEDA
:1021A000A0EB0900371AFEF709FE82462C480068AA
:1021B000C0F3CB307843009045E0701C002842D03B
:1021C000FEF7FCFDA0EB0A00B84200D2A7BB2068D6
:1021D000406820F0E000216848606068B0F5827FC8
:1021E0000DD1A068B0F5004F03D0A068B0F5806FA6
:1021F00005D12068006820F0400021680860A06ACE
:10220000B0F5005F0DD100BF2068006820F40050D9
:10221000216808602068006840F400502168086068
:1022200000BF012084F8510000BF002084F8500056
:1022300000BF0320BDE8F88FFFE7009800B9002732
:102240000098401E0090206880682840A84201D174
:10225000012000E000204045AFD10020EAE7000067
:1022600000000020704710B5FEF7AEFD10BD7047AE
:1022700000BFFEE770B5044615461E46FEF708FB94
:102280002A46334621460320FEF7AAFA18B9FEF77C
:102290009DFA002070BDFEF799FA4FF0FF30F9E784
:1022A00010B501220EA10F4802F06CFE04460D2C61
:1022B00014D14FF400730022114609A002F0B8FABD
:1022C00004465CB9012206A1002002F05BFE044630
:1022D000012203A1034802F055FE0446204610BD2A
:1022E000303A0000A801002030B585B004460D4604
:1022F00000200490009002940395681E04EBC02017
:102300000B49884203D94FF0FF3005B030BDFEF7CE
:10231000BFFA04A96846FEF701FA20B1FEF756FAA3
:102320004FF0FF30F1E7FEF751FA0020EDE7000033
:1023300000F807082DE9F04186B004460D46164620
:102340001F46DDF83080434884420DD100BF42482B
:10235000806940F00400404988610846806900F0C7
:102360000400019000BF6AE03C4884420DD100BFE8
:102370003948806940F0080037498861084680691B
:1023800000F00800019000BF59E0354884420DD1AB
:1023900000BF3148806940F010002F49886108462D
:1023A000806900F01000019000BF48E02D48844291
:1023B0000DD100BF2848806940F02000264988617F
:1023C0000846806900F02000019000BF37E02648F1
:1023D00084420DD100BF2048806940F040001E4972
:1023E00088610846806900F04000019000BF26E047
:1023F0001E4884420DD100BF1748806940F080001C
:10240000154988610846806900F08000019000BF8E
:1024100015E0174884420DD100BF0F48806940F491
:1024200080700D4988610846806900F480700190D1
:1024300000BF04E04FF0FF3006B0BDE8F081029528
:1024400003960597CDF8108002A92046FEF710FBF1
:102450000020F1E70008014000100240000C01409C
:10246000001001400014014000180140001C014010
:102470000020014070B505460E461446012C04D1DB
:1024800031462846FEF794FC04E0002231462846F7
:10249000FEF78EFC70BD000070B504460D46012CA1
:1024A00000D170BD022C00D1FBE7032C05D12A46D8
:1024B0004FF400410248FEF77BFC00BFF1E700004B
:1024C0000008014010B50446012C05D10B48FFF768
:1024D00011F908B1A01E10BD022C05D10848FFF764
:1024E00009F908B1E01EF6E7032C05D10548FFF70E
:1024F00001F908B1201FEEE70020ECE7680000209A
:10250000C00000201801002010B50446012C01D1A4
:10251000801E10BD022C01D1E01EFAE7032C2ED143
:1025200019480078012801D10020F2E7174818491E
:10253000086030211648C16100218160416101615C
:10254000C1600162416281620721C1624FF4007182
:1025500081614FF482700E4948600846FFF7CAF85F
:1025600010B14FF0FF30D4E70948FFF779F910B107
:102570004FF0FF30CDE701200349087002E04FF033
:10258000FF30C6E70020C4E70F000020003C0040F9
:102590001801002013B582B00446012C02D100209E
:1025A00004B010BD022C01D10020F9E7032C11D199
:1025B00000BF0A4890F851000128FAD1012301AA6E
:1025C00003A90648FFF7ACFB00BF044890F8510090
:1025D0000128FAD19DF80400E2E70000180100206C
:1025E0000246012A01D1801E7047022A01D1D01E65
:1025F000FAE7032A3AD181B91F480068006820F041
:1026000038001D4B1B6818601B480068006840F0CC
:102610000800194B1B6818602BE0012910D11648DF
:102620000068006820F03800134B1B6818601248DF
:102630000068006840F020000F4B1B68186018E02D
:10264000022910D10C480068006820F038000A4BBD
:102650001B68186008480068006840F03000064BAE
:102660001B68186005E04FF0FF30BDE74FF0FF300A
:10267000BAE70020B8E700001801002000B58FB0CD
:1026800014210AA8FDF79DFD28216846FDF799FD54
:102690000120009000040190002003900490069017
:1026A000102005900020029002200790C10308919D
:1026B0004FF4E01109916846FEF7EAFD08B100BF4A
:1026C000FEE70F200A9002200B9000200C900E9045
:1026D0004FF480600D9002210AA8FEF741FC08B17A
:1026E00000BFFEE70FB000BD08B5FEF779FBFFF7AE
:1026F000C5FF00BF1248C06940F080501049C86152
:102700000846C06900F08050009000BF00BF00BFC5
:102710000846806940F0010088610846806900F041
:102720000100009000BF00BF00BF0649486820F0CC
:10273000E06040F00070486000BF002008BD00006D
:1027400000100240000001402DE9F04FADF5317D51
:1027500082468B4617469946DDF8E882002500261A
:1027600000202390802103A8FDF72BFDBAF1000F74
:102770000DD05046FDF74CFD48B1BBF1000F06D01F
:10278000B8F1000F03D017B1B9F1000F05D14FF028
:10279000FF300DF5317DBDE8F08F00240EE057F8D5
:1027A000240038B157F82400FDF732FD10B159F874
:1027B000240010B94FF0FF30EBE7641CBB98844253
:1027C000EDDB0122514625A802F006FCB090B0983E
:1027D00010B16FF00100DCE70024F2E0E1E025AA8F
:1027E000802103A801F0A4FE2490249888B9289998
:1027F0002A98884201D1012000E0002018B1002071
:1028000048F82400D7E025A801F081FE6FF002000F
:10281000BFE7002600250EE0FDF7B6FC006803A91F
:10282000495D405C00F0010020B903A8405D03A9A8
:102830008855761C6D1C03A8FDF7EAFCA842EBD86E
:10284000002003A988559DF80C00232800D1A8E09A
:102850005BF8241003A8FDF7BFFC58B19DF80C00ED
:102860005B2807D103A8FDF7D3FC401E03A9085C31
:102870005D2800D095E088E025AA802103A801F01A
:1028800057FE2490249888B928992A98884201D123
:10289000012000E0002018B1002048F824007EE06C
:1028A00025A801F034FE6FF0020072E70026002533
:1028B0000EE0FDF769FC006803A9495D405C00F08B
:1028C000010020B903A8405D03A98855761C6D1C42
:1028D00003A8FDF79DFCA842EBD8002003A988556A
:1028E0009DF80C00232800D14FE0002508E003A844
:1028F000405D232803D1002003A9485505E06D1C45
:1029000003A8FDF785FCA842F1D800BF57F82410B2
:1029100003A8FDF761FC38B33D2103A8FDF76EFC69
:1029200010B33D2103A8FDF769FC02900298401CFA
:1029300002900298FDF76CFC58F82410884205D9E3
:1029400025A801F0E4FD4FF0FF3022E70298FDF7E3
:102950005FFC019059F82400DDE90121FDF718FC26
:102960002398401C23901AE09DF80C005B280BD1A3
:1029700003A8FDF74DFC401E03A9085C5D2803D1A8
:10298000002048F824000AE000BF28992A988842CD
:1029900001D1012000E0002000283FF46DAF00BF0E
:1029A00009E028992A98884201D1012000E00020FE
:1029B00000283FF414AF00BF002125A801F0E0FD7E
:1029C000641CBB988442FFF609AF25A801F09FFD67
:1029D0002398DEE62DE9FF4FADF2DC5D0F461D4684
:1029E0000DF5C26898E80007802140A8FDF7E9FBD3
:1029F000802120A8FDF7E5FBDDF8DC0570B1DDF8EE
:102A0000DC05FDF705FC48B1DDF8E40530B1B9F1AE
:102A1000000F03D015B1B8F1000F05D14FF0FF3012
:102A20000DF2EC5DBDE8F08F00240EE055F82400B7
:102A300038B155F82400FDF7EBFB10B158F824002D
:102A400010B94FF0FF30EBE7641C5445EEDB022F6A
:102A500002DD4FF0FF30E3E70122ECA8DDF8DC15E2
:102A600002F0BAFA8346BBF1000F02D06FF001000A
:102A7000D6E7DDF8DC05FDF7CBFB02461F9020A86A
:102A8000DDF8DC15FDF784FBDDF8DC05FDF7C0FBA8
:102A900020A930220A54132261A802F09DFA83462D
:102AA000BBF1000F02D06FF00100B9E74FE1ECAAD3
:102AB000802140A801F03CFD60906098A0B9EF999A
:102AC000F198884201D1012000E0002000B148E1E6
:102AD00061A801F01CFDECA801F019FD20A802F08E
:102AE00061FD6FF002009BE700260AE0FDF74CFB5A
:102AF000006840A9895D405C00F0010000B105E07C
:102B0000761C40A8FDF784FBB042EFD800BF40A878
:102B1000805D232804D161A940A802F069FB16E179
:102B200061A940A802F064FB40A8DDF8E415FDF7B8
:102B300053FB00287CD0B0E0ECAA802140A801F033
:102B4000F7FC60906098A0B9EF99F198884201D1A4
:102B5000012000E0002000B1A9E061A801F0D7FC4D
:102B6000ECA801F0D4FC20A802F01CFD6FF00200DC
:102B700056E700260AE0FDF707FB006840A9895DDB
:102B8000405C00F0010000B105E0761C40A8FDF7B4
:102B90003FFBB042EFD800BF40A8805D232804D19E
:102BA00061A940A802F024FB77E09DF800015B28B2
:102BB00029D140A8FDF72CFB401E40A9085C5D28E8
:102BC00021D1DFB980216846FDF7FBFA002412E02D
:102BD00059F8240070B1002049F8240058F8243036
:102BE00055F8242069A1684600F06EFC61A968468A
:102BF00002F0FEFA641C5445EADB00BF61A940A85C
:102C000002F0F6FA53E0EFB9002413E055F824106F
:102C100040A8FDF7E1FA60B1002049F8240058F817
:102C2000243055F8242059A140A800F04DFC03E0C1
:102C30005FE0641C5445E9DB00BF61A940A802F0D5
:102C4000D7FA29E0012F0CD1002407E055F8241011
:102C500040A8FDF7C1FA00B102E0641C5445F5DB61
:102C60001AE0022F18D100240FE055F8241040A8D4
:102C7000FDF7B2FA40B158F8243055F8242043A1AA
:102C800040A800F021FC02E0641C5445EDDB00BFCD
:102C900061A940A802F0ACFA00BFEF99F198884210
:102CA00001D1012000E0002000283FF445AF00BF23
:102CB000EF99F198884201D1012000E00020C8B1CD
:102CC000C7B9002412E059F8240070B1002049F877
:102CD000240058F8243055F824202CA140A800F0F6
:102CE000F3FB61A940A802F083FA641C5445EADBB7
:102CF00037E02CE020E0ECAA802140A801F018FC8D
:102D000060906098A0B9EF99F198884201D10120B4
:102D100000E0002000B118E061A801F0F8FBECA889
:102D200001F0F5FB20A802F03DFC6FF0020077E611
:102D300061A940A802F05CFAEF99F198884201D1AC
:102D4000012000E000200028D5D000BF00BFEF998F
:102D5000F198884201D1012000E0002000283FF4D2
:102D6000A6AE00BF61A801F0D2FBECA801F0CFFB3A
:102D7000DDF8DC0502F016FC834620A8DDF8DC1542
:102D800002F022FB834600204AE600002573203D26
:102D90002025730D0A00000010B5012000F0FDF998
:102DA000FF2000F001FA10BD70B505460122002198
:102DB000092000F0B6F9044624B91021284600F095
:102DC0005BF90446FFF7E8FF0CB1012070BD00205D
:102DD000FCE770B505464FF6FF7401E0601E84B253
:102DE000FF2000F0E1F9A84201D0002CF6D10CB987
:102DF000FF2070BD0020FCE77FB56846FFF7D4FFD9
:102E000010B1002004B070BD9DF8000000F0C000BB
:102E1000402809D19DF809009DF8081000EB012019
:102E2000401C84B2A50220E09DF8050000F00F00D0
:102E30009DF80A1000EBD1109DF8091001F0030174
:102E400000EB4100861C9DF8080080119DF80710DA
:102E500000EB81009DF8061001F0030100EB8120DA
:102E6000441CA6F1090004FA00F52846CAE7000050
:102E7000F8B50320FFF748FB012000F08EF902208F
:102E800000F099F9002505E0FF2000F08DF90446D7
:102E9000681C85B2642DF7DB142600BF9522002143
:102EA000084600F03EF90446012C04D0301EA6F17D
:102EB00001018EB2F2D1002051490870012C4AD193
:102EC00087224FF4D571082000F02BF9012847D153
:102ED000002506E0FF2000F067F90DF80500681CEA
:102EE00085B2042DF6DB9DF80200012879D19DF80A
:102EF0000300AA2875D14FF6FE7600BF01220021FB
:102F0000372000F00EF901229107292000F009F97D
:102F1000044624B1301EA6F101018EB2EED1002E7E
:102F20005FD0012200213A2000F0FBF8002858D1A0
:102F3000002506E0FF2000F037F90DF80500681CB9
:102F400085B2042DF6DB9DF8000000F0400018B1BA
:102F500006202B49087044E004202949087040E00D
:102F600001220021372000F0DCF801220021292075
:102F700000F0D7F80446012C17DC02202049087025
:102F80004FF6FE7600BF01220021372000F0C9F87D
:102F900001220021292000F0C4F80446BCB1301EF3
:102FA000A6F101018EB2EED111E0012014490870A2
:102FB0004FF6FE7600BF01220021104600F0B1F866
:102FC000044624B1301EA6F101018EB2F3D12EB118
:102FD00001225102102000F0A4F810B1002008498D
:102FE0000870FFF7D9FE002000F0E5F804480078EB
:102FF00008B10020F8BD0CB12046FBE7AA20F9E794
:10300000100000202DE9F04106460F4615461948EC
:103010000078062800D07F02012D0CD1012239460C
:10302000112000F07EF80446FCB96902304600F039
:1030300023F8044619E001223946122000F071F805
:10304000044600BF4FF40071304600F015F8044606
:1030500006F50076681EC0B2051E01D0002CF1D026
:10306000012200210C2000F05CF8FFF795FE2046BD
:10307000BDE8F0811000002070B504460D46FE202A
:10308000FFF7A7FE08B1012070BD04E0FF2000F0AB
:103090008BF82070641C281EA5F101018DB2F5D1BA
:1030A000FF2000F081F8FF2000F07EF80020EBE721
:1030B00010B5002000F071F800F084F808B9002085
:1030C00010BDFFF769FE0120FAE72DE9F041064641
:1030D0000D4600F077F8074617B10120BDE8F081F2
:1030E000284600F061F8FD2D19D0002404E0305D81
:1030F00000F05AF8601C84B2B4F5007FF7DBFF20C3
:1031000000F052F8FF2000F04FF8FF2000F04CF8DC
:10311000074607F01F00052801D00220DEE7002047
:10312000DCE72DE9F04105460C4617464FF0000854
:10313000FFF732FEFFF7BCFF10B1FF20BDE8F081C2
:1031400045F0400000F030F8200E00F02DF8C4F3F8
:10315000074000F029F8C4F3072000F025F8E0B29A
:1031600000F022F8384600F01FF80C2D02D1FF20A5
:1031700000F01AF84FF01F0800BFFF2000F014F80D
:10318000064606F0800030B1B8F10000A8F1010158
:1031900001F0FF08F1D13046D0E710B504462146D2
:1031A0000320FFF779F910BD10B50446214603202E
:1031B000FFF7F0F910BD10B5044621460320FFF7D4
:1031C0000FFA10BD70B5002400BFFF20FFF7ECFF21
:1031D0000546FF2D01D1002070BD641C6FF07F40BB
:1031E000B4FBF0F100FB114028B90320FFF78CF984
:1031F0000120FFF7D2FF6FF070408442E5D3012039
:10320000EAE700002DE9F04106460F461546204842
:103210000078062800D07F02012D0CD1012239460A
:103220001820FFF77EFF04466CBBFE213046FFF7F7
:103230004CFF044627E016480078012809D00122F7
:1032400000213720FFF76DFF012229461720FFF7E5
:1032500068FF012239461920FFF763FF044694B93D
:1032600000BFFC213046FFF730FF044606F500762C
:10327000681EC0B2051E01D0002CF2D0FD21002036
:10328000FFF723FF0446FFF787FD2046BDE8F081E6
:1032900010000020F0B5ADF5197D002600251421A1
:1032A00006A8FCF78EFF314F3148059006A8049020
:1032B000002003902F48007801284FD100BFE02163
:1032C0002D48FFF711F8B0F1FF3FF8D000BF012201
:1032D0002A490EA801F080FE0446002CF7D116E022
:1032E00000210C910D910BAB08220CA90EA801F046
:1032F00095FF0446204901EBC500DDE90C23FEF7EC
:10330000B9FF6D1C0B98082801D204B908E0119987
:103310001398884201D1012000E000200028DFD06E
:1033200000BF0EA801F0F3F8002215A106A800F0D6
:10333000CBF806A8FCF76CFF0390012003A904AAB0
:1033400005ABCDE9002102903A4602210D48FFF776
:1033500041FB064616B9002006490870054800786A
:1033600008B900F073F80DF5197DF0BD1B000020C1
:103370002B0000203600002000000108E0030020A0
:1033800025640000FA6A000810B58CB000241421EE
:1033900007A8FCF716FF2648069026480590264801
:1033A00004901F2003900220034601220821009070
:1033B0002248FEF7BFFF012208212048FFF75AF8F4
:1033C000012003A904AB05AACDE9001006A91C48F9
:1033D000FFF7BAF90446012C01D1039818B94FF050
:1033E000FF300CB010BD07A80490132003901548BF
:1033F0000590012003A904AB05AACDE9001006A998
:103400000F48FFF7A1F90446012C01D1039810B928
:103410004FF0FF30E5E707A8FCF701FF18B10120E6
:103420000949087002E00020074908700020D8E729
:103430001B00002023000020E003002000180140B2
:10344000FA6A00082B0000203600002008B500248E
:103450001948009008211948FDF732FA0320FFF7B8
:1034600031F8FDF743FE00204FF0E021086148618C
:103470008861012080F3108800BF00BF08E04FF092
:10348000FF310F4840F824100E4840F82410641C07
:10349000082CF4D3002080F3108800BF0098456802
:1034A0000099086880F3088800BF002080F3148822
:1034B00000BFA84700BFFEE7000001080018014058
:1034C00080E100E080E200E00FB4084B10B504A9F1
:1034D00002AA039800F03CF8044602A9002000F07C
:1034E00013F9204610BC5DF814FB000009370008F2
:1034F00002480068C0F30220704700000CED00E0B5
:1035000010B5002804DB0A07130E054A135406E021
:103510000A07140E034A00F00F031B1FD45410BDFA
:1035200000E400E018ED00E0004870474000002093
:1035300002E008C8121F08C1002AFAD1704770477C
:10354000002001E001C1121F002AFBD170470000DA
:103550002DE9FF4F8BB09A460F460546002606E040
:1035600025280BD052460D9990476D1C761C287863
:103570000028F5D10FB03046BDE8F08F0024A046FA
:103580000122604900E0044315F8013F203B02FAA4
:1035900003F00842F7D128782E2817D115F8010F2B
:1035A00044F004042A280ED06FF02F022878A0F1EE
:1035B000300109290AD808EB880102EB410100EB30
:1035C00001086D1CF2E757F8048B6D1C28786928F8
:1035D0003ED006DC0028CDD063280BD0642804D16F
:1035E00036E0732810D075284BD052460D9990477D
:1035F000761C85E017F8040B8DF8000000208DF88C
:103600000100E946012003E057F8049B4FF0FF302A
:1036100061074FF0000401D40AE0641C44450DDA50
:103620008442FADB19F804100029F6D106E0641C84
:103630008442FCDB19F804100029F8D1264404E088
:1036400019F8010B52460D999047641EF8D257E0C5
:1036500001CF4FF00A0B002802DA40422D2102E090
:10366000210504D52B218DF82410012103E0E10769
:1036700005D02021F7E70DF1200908910CE0002189
:10368000F9E701CF4FF00A0BF9E75946FCF7D4FDF3
:1036900001F1300209F8012D0028F6D1ADEB090047
:1036A00000F1200B600701D44FF00108D84502DD7E
:1036B000A8EB0B0000E000208046002406E009A8EB
:1036C0005246005D0D999047641C761C0898844210
:1036D000F5DB04E0302052460D999047761CB8F196
:1036E0000001A8F10108F5DC05E019F8010B5246CC
:1036F0000D999047761CBBF10001ABF1010BF4DC96
:103700006D1C34E7092801000A68531C0B60107017
:10371000704700002DE9F041044688460020E07023
:10372000401E60634146204602F0F4FC10B10420C4
:10373000BDE8F08104F2362002F021FB074694F840
:103740003850EB2D03D0E92D01D0E82D34D14AF6C5
:103750005520874208D108221BA104F18A0002F0FB
:103760005BFB08B90020E3E704F1430002F007FB2C
:103770000646701E3040F8B9B6F5007F1CDBB6F582
:10378000007F19DC4520055DB5B1681E284098B959
:103790004820005D012803D04820005D02280BD19D
:1037A00004F1490002F0EBFA30B104F14E0002F0EE
:1037B000E6FA08B10020BBE74AF65520874201D15E
:1037C0000220B5E70320B3E74641543332202020DE
:1037D00000000000024600E0521C107810B1107882
:1037E0008842F9D110787047F0B503460D461E683F
:1037F000986A021D680A7789B0FBF7F400BF02CA15
:1038000009B90020F0BD8C4200D202E0641A121DFA
:10381000F5E700BF10682044F4E70246891ED0692E
:10382000801E884201D8002070475389106B03FB2B
:103830000100F9E72DE9F04780460C4604F11A0033
:1038400002F09DFA10B10020BDE8F087207800F06A
:103850003F00401E00EB800101EBC0054FF0010965
:10386000002621E01849895D081902F088FA074608
:10387000B9F1000F11D0FF2D0BD8384602F03AF8FD
:10388000824629466D1C38F8110002F033F8824553
:1038900001D00020D8E7B94605E04FF6FF70874217
:1038A00001D00020D0E7761C0D2EDBD3207800F06D
:1038B000400038B1B9F1000F04D038F8150008B154
:1038C0000020C1E70120BFE7906600082DE9F0471E
:1038D00082468846DAF80040B8F1000F06D1276921
:1038E00017B1E069B84215D8012713E041465046A8
:1038F00002F088F90546022D02D20120BDE8F087CA
:10390000681C08B92846F9E7E069A84201D92846A9
:10391000F4E74746606908B90020EFE7002647450D
:1039200018D17E1CE069B04200D8022631465046CC
:1039300002F068F90546012D01D0681C08B9284637
:10394000DCE73DB12569022D03D3E069A84200D927
:103950002F460026E6B93E4600BF761CE069B0421D
:1039600004D80226BE4201D90020C7E7314650469E
:1039700002F048F9054605B909E0012D01D0681C9F
:1039800008B92846BAE7BE42E7D10020B6E700BF33
:103990004FF0FF323146204602F01CFC8146B9F15F
:1039A000000F08D1B8F1000F05D03246414620463D
:1039B00002F010FC8146B9F1000F0DD12661E069DB
:1039C000801E6169814202D86069401E6061207971
:1039D00040F00100207107E0B9F1010F02D14FF072
:1039E000FF3000E001200646304687E72DE9F34F1F
:1039F00083B08146049800680090D9F80000C76839
:103A0000002500BF684602F0F2FD02900298401CBB
:103A100018B9062005B0BDE8F08F0298B0F5803FD8
:103A200005D30298020C28466D1C27F81020029836
:103A300084B2202C03DB2F2C01D05C2C00D111E0B0
:103A4000802C06DA214693A0FFF7C4FE08B10620B9
:103A5000E0E7FF2D01D30620DCE728466D1C27F8A0
:103A60001040CFE700BF202C01DA04260CE000262E
:103A700002E00098401C0090009800782F28F8D0B1
:103A8000009800785C28F4D0009904980160012D1A
:103A900004D1681E37F810002E280BD0022D24D137
:103AA000681E37F810002E281FD1A81E37F8100006
:103AB0002E281AD1002027F8150080460AE0A845D4
:103AC00001D22E2100E0202109F1200000F8081089
:103AD00008F10108B8F10B0FF1D346F0200109F10C
:103AE000200000F80810002094E708E0681E37F86E
:103AF0001040202C02D02E2C00D002E06D1E002D94
:103B0000F4D100BF002027F815000DB9062081E789
:103B10004FF0000A01E00AF1010A37F81A002028E4
:103B2000F9D0BAF1000F03D137F81A002E2801D1CD
:103B300046F0030600E06D1E25B1681E37F8100040
:103B40002E28F8D10B22202109F1200002F083F960
:103B50004FF00008C3460820019000BF50460AF10C
:103B6000010A37F8104004B968E0202C03D02E2C4D
:103B700004D1AA4502D046F00306EFE7019880453C
:103B800001D2AA4516D101980B2802D146F00306AE
:103B900054E0AA4501D046F00306AA4500D94DE0FD
:103BA000AA464FF008080B2001904FEA8B604FEABD
:103BB000106BD3E7802C0EDB46F0020640F2B51105
:103BC000204601F077FE044604F0800018B104F0AE
:103BD0007F0033490C5CFF2C10DD0198401E4045EE
:103BE00004D846F00306DDF80480B7E72212404609
:103BF00008F1010809F120010A5418E024B1214616
:103C000028A0FFF7E7FD18B15F2446F003060EE099
:103C1000412C03DB5A2C01DC4BF0020B612C06DB40
:103C20007A2C04DC4BF0010BA4F1200084B2404656
:103C300008F1010809F120010C548FE700BF99F841
:103C40002000E52802D1052089F8200001980828E5
:103C500003D14FEA8B604FEA106B0BF00C000C287D
:103C600003D00BF00300032801D146F0020606F052
:103C7000020048B90BF0010008B146F010060BF045
:103C8000040008B146F008062B2000F80960002067
:103C9000C0E60000222A3A3C3E3F7C7F0000000044
:103CA0009D6600082B2C3B3D5B5D00002DE9FF4F1E
:103CB00085B09A4603AA0121059800F0C1FB18B10E
:103CC000012009B0BDE8F08FDDF80C904FF03F08FF
:103CD000082701E07806070E37B1B9FBF7F0B0FB13
:103CE000F8F0B0F5806FF5D807B9FF274FF40072F0
:103CF0000021504602F0AFF80AF5DF764FF0000BD6
:103D0000444669E0069850F82B50642D07D801D13D
:103D1000484603E06420B9FBF0F0684305466019AB
:103D2000484501D8601901D3A9EB040505B959E04C
:103D3000214606F1080002F0CAFB294606F10C00F4
:103D400002F0C5FB07983071B4FBF8F0B0FBF7F058
:103D50000490B4FBF8F0B0FBF7F107FB1100C0B220
:103D60000290B4FBF8F008FB1040401CC0B2019078
:103D700002987070C021049801EA900001990843EC
:103D8000B0700498F0706019401EB0FBF8F0B0FB02
:103D9000F7F004906019401EB0FBF8F0B0FBF7F1AB
:103DA00007FB1100C0B202906019401EB0FBF8F191
:103DB00008FB1100401CC0B2019002987071C02134
:103DC000049801EA900001990843B0710498F071D9
:103DD00010360BF1010B2C44BBF1040F02D20CB1D5
:103DE0004C458FD300BF4AF655210AF5FF7002F00B
:103DF0007AFB012300225146059800F072FB08B1BE
:103E000001205EE700205CE7014609B10020704711
:103E10000020FCE7014609B1002070470020FCE7C4
:103E20002DE9F04104460E46D4F8008000212046DA
:103E300000F0A6FA0546EDB9002700BF4046A1698B
:103E400002F068F9054605B113E0E0690078E5285D
:103E500002D0E069007820B9781C0746B04201D151
:103E600007E000270121204600F0EBF80546002D71
:103E7000E4D000BF042D00D107252846BDE8F0811D
:103E80002DE9F04704468946204602F08BFB10B12D
:103E90000120BDE8F08749462046FFF7BEFC0746F3
:103EA00067634FF40072002104F1380001F0D3FF82
:103EB00060894FF40041B1EB402F01D8084601E082
:103EC0006089400206464FF0000800E07608B6F52B
:103ED000007F05D9304601F0CAFCB0F10008F5D0EA
:103EE000B6F5007F17D932460021404601F0B3FFF6
:103EF000760A002500E035446089A84207D97A197E
:103F000060783346414600F0ECFA0028F3D0404692
:103F100001F0B3FC10E004F138080126002500E0B0
:103F200035446089A84207D97A19607833464146FA
:103F300000F0D7FA0028F3D06089A84201D0012010
:103F4000A7E70020A5E72DE9F0470446D4F800A034
:103F50000021204600F014FA064616B13046BDE8AE
:103F6000F0874FF0FF08C1464FF0FF30E06200BF1E
:103F70005046A16902F0CEF8064606B15EE0E0695F
:103F800005780DB9042659E0E069C07A00F03F07D2
:103F9000A771E52D04D007F0080038B10F2F05D028
:103FA0004FF0FF084FF0FF30E06240E00F2F22D1CA
:103FB0002B20005D00F0400098BB05F0400038B1B8
:103FC000E06990F80D9005F0BF05A8462069E06211
:103FD00045450CD1E069407B484508D1E169DAF8F4
:103FE0000C00FFF727FC10B1A8F1010000E0FF2052
:103FF00000F0FF081BE0B8F1000F05D1E06902F006
:1040000078FA484500D119E02B20005D00F001004E
:1040100040B90B2204F12001E06901F0FDFE08B96E
:104020000CE004E04FF0FF084FF0FF30E0620021A9
:10403000204600F006F80646002E99D000BF304614
:104040008DE72DE9F041044688462768206900F194
:104050002006B6F5001F01D30020A061A06910B9A9
:104060000420BDE8F081C6F30800002845D1A0690E
:10407000401CA061606938B93889B0EB561F3CD844
:104080000020A0610420ECE77889401E00EA562059
:1040900098BB2046616901F0B5FD0546012D01D8A8
:1040A0000220DEE7681C08B90120DAE7F869A842B7
:1040B0001DD8B8F1000F03D10020A0610420D0E783
:1040C00020466169FFF702FC05460DB90720C8E7E5
:1040D000012D01D10220C4E7681C08B90120C0E706
:1040E00029463846FFF7CCFE08B10120B9E76561E3
:1040F00029463846FFF791FBA0612661C6F3080107
:1041000007F138000844E0610020AAE72DE9F05FDC
:10411000044689460426D4F800A04FF0FF08C346A1
:1041200053E05046A16901F0F5FF064606B14FE0A5
:10413000E06905780DB904264AE0E069C07A00F02C
:104140003F07A771E52D0AD02E2D08D027F02000BB
:10415000082801D1012000E00020484502D04FF09E
:10416000FF082BE00F2F1DD105F0400038B1E069AA
:1041700090F80DB005F0BF05A8462069E0624545FE
:104180000CD1E069407B584508D1E169DAF80C00B0
:1041900001F0DAFF10B1A8F1010000E0FF2000F00B
:1041A000FF080BE0B8F1000F04D1E06902F0A1F9BB
:1041B000584502D04FF0FF30E06209E00021204670
:1041C000FFF73FFF064606B102E0A0690028A8D12C
:1041D00000BF0EB10020A0613046BDE8F09F2DE980
:1041E000FE4F044626682B20005D00F0A00010B1B1
:1041F0000620BDE8FE8F4FF0000901E009F101093A
:10420000F06830F819000028F8D10C2204F12001E0
:10421000684601F013FE9DF80B0000F0010028B382
:1042200040212B2001554FF001080EE0434669461E
:1042300004F12000F26801F07FFC2046FFF783FEC6
:10424000054605B104E008F10108B8F1640FEDD3AB
:1042500000BFB8F1640F01D10720CAE7042D01D0D7
:104260002846C6E79DF80B102B2001559DF80B0042
:1042700000F0020030B109F10C000D21B0FBF1F0AB
:10428000401C00E00120074639462046FFF7C8FDE4
:1042900005464DBB781E071E26D02069A0EB4711AE
:1042A000204600F06DF80546F5B904F1200002F053
:1042B00020F9824600BF3046A16901F02BFF054678
:1042C00005B110E0FAB2E1695346F06802F01EF859
:1042D0000120F07000212046FFF7B3FE054615B916
:1042E000781E071EE7D100BFC5B93046A16901F0AD
:1042F00011FF054695B920220021E06901F0ABFDD0
:104300000B2204F12001E06901F098FD2B20005DF3
:1043100000F01800E16908730120F070284668E792
:104320002DE9F041044626682769E06A401C08B977
:10433000002003E02046E16A00F022F80546E5B9D6
:1043400000BF3046A16901F0E5FE054605B110E069
:1043500000BFE520E16908700120F0702069B842D3
:1043600000D306E000212046FFF76BFE0546002D36
:10437000E7D000BF042D00D102252846BDE8F0811A
:104380002DE9F04104460D462668B5F5001F02D21E
:1043900005F01F0010B10220BDE8F0812561A7687B
:1043A0001FB93078032800DBF76A47B93089B0EBD2
:1043B000551F01D80220EFE7F06AA0611CE0708968
:1043C0004FEA402811E03946204601F01BFC074621
:1043D000781C08B90120DFE7022F02D3F069B84248
:1043E00001D80220D8E7A5EB08054545EBD23946B0
:1043F0003046FFF712FAA0616761A06908B9022090
:10440000CAE7A06900EB5520A061C5F3080106F1D9
:1044100038000844E0610020BEE770B5054665B984
:10442000FEF726FD044634B10020FEF7C4FEFF204F
:10443000FEF7BAFE01E0002070BD00BF0120FBE7DF
:104440002DE9F04106460F4615462EBB37B1012F28
:104450001AD0022F0FD0032F1BD111E00020FEF73E
:104460009CFEFEF7AFFE08B9002400E00124012005
:10447000FEF793FE0FE04FF40070288000240AE05E
:1044800008202880002406E0FEF7B6FC28600024FF
:1044900001E0042400BF00E001242046BDE8F081D3
:1044A0002DE9F04106460F4690461C4614B90420FB
:1044B000BDE8F0816EB9E2B241463846FEF7A2FD92
:1044C000054625B1FF20FEF76FFE0120F0E7002032
:1044D000EEE70420ECE7014609B90020704701200F
:1044E000FCE72DE9F04105460E461746984665B9AA
:1044F00008F0FF0239463046FEF784FE044614B940
:104500000020BDE8F0810120FBE70420F9E738B581
:104510000546284600F0F6FF04463CB969462846A1
:1045200002F08BF804460CB900202860204638BD04
:104530002DE9FC4780460C46914600254646641E00
:1045400013E06B46012201A9484600F067FE00987F
:10455000012800D00BE09DF8047000BF06F8017B35
:104560006D1C0A2F00D102E000BFA542E9DB00BFAD
:104570000020307015B14046BDE8FC870020FBE705
:104580002DE9F04F89B004460D4607A9204602F0F8
:1045900054F80890089808B9607C0890089818B1F9
:1045A000089809B0BDE8F08FA06A00287CD0681C8C
:1045B000002843D1D4F8289059F8040B0290022027
:1045C0000190A76867B300BF03970020049001988B
:1045D000801C019000BF05970498401C0490394648
:1045E000204601F00FFB0746012F02D8022060741D
:1045F000D7E7781C10B901206074D2E70598401CF9
:104600008742E8D0DDE90101884205D8049849F8DD
:10461000040B039849F8040B0798C069B842D3D833
:104620000198A16A0860DDE90101884203D80020F1
:10463000C9F80000FAE011200890F7E0E068A8420D
:1046400000D2E5686561002DF4D0691E2046FFF7B1
:10465000CBF8A061A1690798FFF7DFF88246BAF1AD
:10466000000F02D1022060749BE707984089401E2A
:10467000691E00EA51208244A08AC0F30800002885
:10468000D8D0E0695045D5D0207C00F0800080B1C2
:10469000E26907994878012304F12C01FFF721FF13
:1046A00018B1012060747CE712E0207C00F07F00EC
:1046B0002074079948780123524604F12C01FFF732
:1046C000EFFE10B1012060746BE7C4F81CA0ADE0F0
:1046D000E068A84204D2207C00F0020000B9E5683E
:1046E000606906904FF0000BC4F814B0002D6AD03A
:1046F000079840894FEA4028069890B1681EB0FBA1
:10470000F8F10698401EB0FBF8F0814209D30698F4
:10471000401EA8F101018843606160692D1AA669F5
:1047200012E0A6687EB900212046FFF7CFF80646C2
:10473000012E02D10220607433E7701C10B90120F1
:1047400060742EE7A660A661D6B325E0A5EB080548
:10475000606940446061207C00F0020040B100BF0D
:1047600031462046FFF7B2F8064636B9002515E077
:104770003146204601F046FA0646701C10B9012069
:1047800060740EE7012E03D90798C069B04202D8C1
:104790000220607405E7A6614545D7D800BF60696F
:1047A00028446061C5F3080050B131460798FFF70F
:1047B00034F88346BBF1000F03D102206074F0E6A9
:1047C00001E00BEB552BE1686069884205D960690F
:1047D000E060207C40F040002074A08AC0F3080014
:1047E00020B3E069584521D0207C00F0800078B1EA
:1047F000E26907994878012304F12C01FFF771FE63
:1048000010B101206074CCE6207C00F07F002074A1
:104810000799487801235A4604F12C01FFF740FE1E
:1048200010B101206074BCE6C4F81CB00898B8E66A
:104830002DE9FF4F99B00F46154619A801F056FA19
:1048400003900398002803DA0B201DB0BDE8F08F19
:10485000FC49039851F8200028B10021F94A039837
:1048600052F8200001700398C0B2169000201590F5
:1048700007B9F54F1698FFF7D0FD0290029800F0A7
:10488000010008B10320E0E7029800F0040008B13D
:104890000A20DAE778681390139838B913AA03212D
:1048A0001698FFF7CDFD08B101201390139840B181
:1048B0001398B0F5004F04D81398401E1399084080
:1048C00008B1012013904FF40079387800F00F0000
:1048D00018907878012804DB7878022801DC787851
:1048E00000E001200690B96889B1B968B1F5004FC0
:1048F0000DD848464FEAE97109EBD1614911BA6810
:10490000B2FBF1F301FB132109B9B96801E04FF4DF
:1049100000710591F868B0F1807F05D8F868411EF4
:10492000084008B9F86800E0002007900798B0FB3D
:10493000F9F007901C98B0FBF9F01490149808B99E
:10494000112082E72C462CB9149901FB09F000F0E4
:104950008EFF04460CB9112077E7002011901090CB
:1049600000BF11AA01211698FFF76AFD28B115B9F9
:10497000204600F082FF012067E7189800F0080049
:1049800040B911983F2805D93F201090DDE910016A
:10499000081A11901198802805D215B9204600F008
:1049A0006CFF0E2051E700BF00BF0798802801D997
:1049B00080200790189800F0020030B1189800F09D
:1049C000010010B94FF003080CE0189800F0010046
:1049D00028B915B9204600F050FF132035E74FF0F5
:1049E000020800BF00BF00BF079EB8F1030F31D11E
:1049F000A6B911984FEA504B00200490012603E01D
:104A00000498401C049076009049049831F81000F6
:104A100020B1049831F810005845F1D91198B0FB35
:104A2000F6FA082000EB8A004844401EB0FBF9F07B
:104A3000099020200A90002008904FF6F5708245DA
:104A400002D9834882453BD915B9204600F015FFAD
:104A50000E20FAE6A6B911984FEA103B0020049008
:104A6000012603E00498401C0490760079490498DC
:104A700031F8100020B1049831F810005845F1D9F0
:104A80001198B0FBF6FA40F6F570824503D9042080
:104A900000EB4A0B07E04FF001080AEB4A00401C0C
:104AA000032101EB500B0BEB0900401EB0FBF9F0AA
:104AB000099001200A9005984001B0FBF9F0089098
:104AC0000A99109808440F90069A09990F9801FBCB
:104AD0000201089808440E9013990E980844401E4D
:104AE000491E20EA01010E98A1EB000BB8F1030F5B
:104AF00006D10A9858440A900F9858440F9013E032
:104B00000698BBFBF0F100FB11B038B1ABF1010B23
:104B10000A98401C0A900F98401C0F900698BBFB07
:104B2000F0F10998084409900E9800EB06111098CE
:104B3000081A1199884205D915B9204600F09DFE42
:104B40000E2082E611990A980A1A0699099800FB24
:104B500011210898081AB0FBF6FAB8F1030F0FD12B
:104B60004FF6F57082450BD8079818B97008079072
:104B700000B148E015B9204600F07FFE0E2064E643
:104B8000B8F1020F31D14FF6F57082451CD9079864
:104B900030B94020B0EB460F02D37000079032E0EE
:104BA000189800F0020010B14FF003082BE00798AE
:104BB00020B970000790802800D824E015B920465D
:104BC00000F05BFE0E2040E640F6F57082450CD802
:104BD000079820B970000790802800D813E015B915
:104BE000204600F04AFE0E202FE6B8F1010F09D151
:104BF00040F6F570824505D915B9204600F03DFE16
:104C00000E2022E600E0EFE600BF4A4600212046E3
:104C100001F021F90B2210A1204601F00FF94946BD
:104C200004F10B0001F05FFC66730A9881B204F195
:104C30000E0001F058FC06982074B8F1030F11D152
:104C4000002010E0140000203C6700082C670008DA
:104C5000F5FFFF0F1E670008EBFE904D53444F53C6
:104C6000352E3000059881B204F1110001F03BFCB3
:104C70001198B0F5803F06D2119881B204F113006B
:104C800001F031FC04E004F12000119901F01FFC57
:104C9000F82060753F2104F1180001F024FCFF2189
:104CA00004F11A0001F01FFC04F11C00109901F03E
:104CB0000EFCB8F1030F28D101F014F80146009062
:104CC00004F1430001F003FC04F12400099901F010
:104CD000FEFB022104F12C0001F0F9FB012104F19B
:104CE000300001F000FC062104F1320001F0FBFB72
:104CF000802084F84000292084F84200132294A1E7
:104D000004F1470001F09AF819E000F0EBFF0146CA
:104D1000009004F1270001F0DAFB099881B204F158
:104D2000160001F0E0FB802084F82400292084F89C
:104D3000260013228BA104F12B0001F07FF84AF624
:104D4000552104F5FF7001F0CEFB01232146109A96
:104D50001698FFF7C6FB28B115B9204600F08DFD67
:104D6000012072E5B8F1030F33D10123109A921D8F
:104D700021461698FFF7B5FB4A460021204601F070
:104D80006AF87D49204601F0A2FB7C4904F5F270E7
:104D900001F09DFBAAF1010104F5F47001F097FB0D
:104DA000022104F5F67001F092FB4AF6552104F554
:104DB000FF7001F098FB0123109AD21D214616982E
:104DC000FFF78FFB0123109A521C21461698FFF71C
:104DD00088FB149800FB09F20021204601F03BF803
:104DE0000F980D900020049048E0B8F1030F10D107
:104DF0006FF00701204601F06AFB4FF0FF31201DE4
:104E000001F065FB6FF0704104F1080001F05FFBF9
:104E10000AE0B8F1010F01D1594801E06FF0070035
:104E20000146204601F053FB0998129000BF1499E7
:104E30001298884201D9149800E0129883465B4684
:104E400021460D9A1698FFF74CFB28B115B920465C
:104E500000F013FD0120F8E44A460021204600F04E
:104E6000FAFF0D9858440D901298A0EB0B00129089
:104E700012980028DBD10498401C049006990498ED
:104E80008842B2D3B8F1030F01D1304600E0089850
:104E9000129000BF14991298884201D9149800E02A
:104EA000129883465B4621460D9A1698FFF719FB28
:104EB00028B115B9204600F0E0FC0120C5E40D98AA
:104EC00058440D901298A0EB0B00129012980028F5
:104ED000E0D100BFB8F1030F02D10C2017900DE014
:104EE0001198B0F5803F02D30620179006E0B8F184
:104EF000020F01D1042000E00120179000BF189894
:104F000000F0080090B911980B9000200C902346F7
:104F10000BA9DDE91602FEF7C9FE0190019828B140
:104F200015B9204600F0A9FC01988EE40022114634
:104F30001698FFF785FA28B115B9204600F09DFCB8
:104F4000012082E415B9204600F097FC00207CE4A3
:104F50004E4F204E414D45202020204641543332B3
:104F6000202020004E4F204E414D4520202020463D
:104F70004154202020202000525261417272416130
:104F8000F8FFFF00F7B582B016460398019001A81C
:104F900000F0ACFE0546002D02DA0B2005B0F0BD96
:104FA0000C4850F825400CB100202070029810B138
:104FB0000020029908700749029841F825000EB9AF
:104FC0000020EBE7002202A903A800F04DFF0746EE
:104FD0003846E3E7140000202DE9F74F90B004466F
:104FE00016461CB9092013B0BDE8F08F06F03F0645
:104FF000324603A911A800F037FF0546002D75D1F0
:10500000039804904FF4007000F031FC8346BBF12C
:10501000000F01D11120E6E70398C0F80CB004A8F6
:10502000119900F0FBFC05462DB99DF83B0000F0FE
:10503000800000B1062506F01C00002857D045B1BD
:10504000042D03D104A8FFF7CAF8054646F0080668
:105050000AE09DF8160000F0110008B1072503E0F2
:1050600006F0040000B10825002D51D106F008001B
:1050700000284DD000F036FE01900B9901F10E0092
:10508000019901F024FA0B9901F11600019901F040
:105090001EFA0B99039800F053FE814620200B99CD
:1050A000C87200220B99039801F0FFF90B9901F1E6
:1050B0001C00002101F00BFA01200399C870B9F11E
:1050C000000F25D00398D0F834A00022494604A848
:1050D00001F09EF90546DDB95146039801F01AF832
:1050E0000546A9F101000399086111E07BE07DB953
:1050F0009DF8160000F0100008B1042508E006F045
:10510000020028B19DF8160000F0010000B107254B
:105110004DB906F0080008B146F040060398406B10
:1051200020620B986062002D5AD10B99039800F011
:1051300007FEA0600B9901F11C0000F014FEE06076
:105140000020A062039820600398C088A080267485
:1051500000206074E06160614FF40072002104F18E
:105160002C0000F078FE06F0200058B3E06848B349
:10517000E06860610398408940020290A768D4F813
:105180000C800DE03946204600F03CFD0746012F1B
:1051900000D80225781C00B901250298A8EB000868
:1051A00015B902988045EDD8A7615DB9C8F308002C
:1051B00040B139460398FEF730FB8246BAF1000F42
:1051C00001D102250CE00AEB5820E061E269039965
:1051D0004878012304F12C01FFF762F900B10125A1
:1051E000584600F04AFB0DB1002020602846FAE640
:1051F00030B593B004460D462946684601F0FEF8E6
:1052000004E014F8011B684601F0C0F8207800287B
:10521000F7D1684601F0DCF813B030BD2DE9FF4F3F
:1052200085B0044615469A46DDF818B00020CAF845
:10523000000003A9204601F000FA0490049810B978
:10524000607C049018B1049809B0BDE8F08F207C10
:1052500000F0010008B90720F6E76169E068401A2C
:1052600001900198854200D9019DA8E0A08AC0F371
:105270000800002874D103984089401E616900EA43
:105280005129B9F1000F1FD1606910B9A0680290CF
:105290000CE0A06A28B120466169FEF7A5FA0290E9
:1052A00004E02046A16900F0ADFC029002980228BB
:1052B00002D202206074C7E70298401C10B9012096
:1052C0006074C1E70298A061A1690398FEF7A5FA8E
:1052D000064616B902206074B6E74E444FEA5528D8
:1052E000B8F1000F29D009EB0800039949898842D9
:1052F00003D903984089A0EB0908039948784346ED
:1053000032465946FFF7CCF810B1012060749BE794
:10531000207C00F0800068B1E069801B404509D224
:10532000E169891B0BEB41204FF4007204F12C0161
:1053300000F084FD4FEA482737E0E069B04220D012
:10534000207C00F0800080B1E26903994878012355
:1053500004F12C01FFF7C5F818B10120607473E760
:1053600010E0207C00F07F0020740399487801232E
:10537000324604F12C01FFF793F810B1012060745C
:1053800062E7E661A08AC0F30800C0F50077AF428B
:1053900000D92F46A08AC0F3080204F12C0011188E
:1053A0003A46584600F04AFD00BFED1BDAF800000F
:1053B0003844CAF80000BB44606938446061002D7D
:1053C0007FF454AF00203FE72DE9F341A2B023A8BA
:1053D00000F08CFC022209A922A800F045FD044639
:1053E000002C7DD1099816904FF4007000F03FFA20
:1053F00007461FB9112024B0BDE8F0810998C760A5
:1054000016A8229900F00AFB04462CB99DF88300E7
:1054100000F0A00000B10624002C6ED1202201A8CB
:105420001D9900F00BFD302216A90AA800F006FD18
:105430000AA8239900F0F2FA04465CB918990C986E
:10544000884205D11A990E98884201D1042000E0C3
:1054500008200446042C46D10AA8FEF7C0FE0446E4
:10546000002C40D1119D13220DF1110105F10D0009
:1054700000F0E4FC9DF80F00E872E87A00F01000FC
:1054800018B9E87A40F02000E87201200999C87044
:10549000E87A00F0100030B30C991898884222D0B6
:1054A0002946099800F04CFC804641460998FEF7D1
:1054B000B4F906460EB9022415E03146099800F009
:1054C00029FE0446099800F1580564B968782E2829
:1054D00009D129460C9A099800F0E7FF012000E065
:1054E0000EE00999C87044B916A8FEF719FF0446E2
:1054F0001CB9099801F00EF80446384600F0BDF9D1
:10550000204678E7F8B504466946204601F095F84C
:105510000646002E44D1207C00F0400000283FD0F9
:10552000207C00F0800070B1E26900994878012386
:1055300004F12C01FEF7D5FF08B10120F8BD207C55
:1055400000F07F00207400F0CDFB0746216A009830
:1055500000F0E0FD06461EBB656AE87A40F02000D8
:10556000E8722946A268206800F09FFF05F11C0040
:10557000E16800F0ACFF394605F1160000F0A7FF26
:10558000002105F1120000F0AEFF01200099C87063
:10559000009800F0BFFF0646207C00F0BF0020749A
:1055A0003046CBE771B599B000250222694619A8AB
:1055B00000F05AFC0446002C60D100980D904FF486
:1055C000007000F054F9064616B911201AB070BDEB
:1055D0000098C6600DA8199900F020FA04462CB96D
:1055E0009DF85F0000F0200000B10624002C42D19D
:1055F0009DF85F0000F0800008B1062405E09DF8EA
:105600003A0000F0010000B1072414BB149900987F
:1056100000F096FB05469DF83A0000F01000C0B17E
:1056200000988069A84201D1072412E000980190F7
:105630000395002101A8FEF7A3FE04464CB9002102
:1056400001A8FEF763FD044604B90724042C00D129
:10565000002484B90DA8FEF763FE044634B92DB1C9
:10566000002229460DA800F0D3FE04461CB900987C
:1056700000F050FF0446304600F0FFF82046A5E752
:105680002DE9FF4F83B0044615469B4604980090D1
:105690000020CBF8000001A9204600F0CEFF0290C8
:1056A000029810B9607C029018B1029807B0BDE86A
:1056B000F08F207C00F0020008B90720F6E700BF59
:1056C000606928446169884202D26069C0F1FF358F
:1056D000C3E0A08AC0F3080000287DD1019840896A
:1056E000401E616900EA512ABAF1000F26D16069B3
:1056F00038B9A76897B900212046FEF7E7F80746B2
:105700000CE0A06A28B120466169FEF76DF80746F3
:1057100004E02046A169FEF7D9F8074607B99FE0E3
:10572000012F02D102206074C0E7781C10B901205B
:105730006074BBE7A761A06800B9A760207C00F097
:10574000800078B1E26901994878012304F12C01C5
:10575000FEF7C7FE10B101206074A7E7207C00F0BF
:105760007F002074A1690198FEF757F8064616B924
:10577000022060749AE756444FEA5529B9F1000FA8
:105780002BD00AEB090001994989884203D9019875
:105790004089A0EB0A09019948784B4632460099A6
:1057A000FEF79FFE10B1012060747FE7E069801B67
:1057B00048450ED2E069801B009A02EB40214FF46D
:1057C000007204F12C0000F039FB207C00F07F0017
:1057D00020744FEA49282BE013E0E069B0420FD073
:1057E000E168606988420BD201994878012332460A
:1057F00004F12C01FEF754FE10B10120607455E74E
:10580000E661A08AC0F30800C0F50078A84500D979
:10581000A846A18AC1F3080204F12C01501842469F
:10582000009900F00BFB207C40F08000207400BF4A
:10583000A5EB0805DBF800004044CBF80000009819
:1058400040440090606940446061E168606988425A
:1058500001D9606900E0E068E060002D7FF439AFB5
:1058600000BF207C40F04000207400201EE710B5EF
:105870000446204600F09AFA10BD10B504462046B2
:1058800000F032F910BD000010B502460020084BB0
:10589000802A01DA104609E040F2B514A14205D190
:1058A000FF2A03DCA2F1800433F8140010BD0000CD
:1058B0004C67000810B5024600200D4B802A01D22B
:1058C00090B213E0B2F5803F10D240F2B514A1427D
:1058D0000CD1002001E0441CA0B2802803DA33F888
:1058E00010409442F7D100F18004E0B210BD0000F6
:1058F0004C67000870B5B0F5803F4DD281B2B1F56C
:10590000805F01DA254E00E0254E324600BF32F8B6
:10591000023B0BB1994200DA3CE032F8024B25120F
:10592000E4B21E198E4230DD092D2CD2DFE805F0DD
:1059300005090F13171B1F232700CE1A32F8161064
:1059400021E0CE1A06F001068E1BB1B21BE0A1F1D8
:105950001006B1B217E0A1F12006B1B213E0A1F137
:105960003006B1B20FE0A1F11A06B1B20BE001F1BD
:105970000806B1B207E0A1F15006B1B203E0A1F50B
:10598000E356B1B200BF00BF04E0002DBFD102EB6F
:105990004402BCE700BF084670BD00004C68000828
:1059A0003E6A00082DE9FF4107460D4600213846B2
:1059B000FDF7B0FE0646022E06D0032E00D21DB91A
:1059C000304604B0BDE8F08100BF00240AE007F5CE
:1059D000FB7101EB041101F1080000F0C4F94DF86E
:1059E0002400641C042CF2D30DB1681E00E00020DA
:1059F000044600BF5DF8240028B15DF82410384645
:105A0000FDF788FE00E0032006462DB9022E03D3E1
:105A1000601C04460428EDD33046D2E72DE9F3415B
:105A200004462768019800782F2806D0019800784E
:105A30005C2802D0B869A0600DE002E00198401C2B
:105A40000190019800782F28F8D0019800785C2800
:105A5000F4D00020A06001980078202808D280218E
:105A60002B20015500212046FEF78AFC054637E031
:105A700000BF01A92046FDF7B9FF054605B12EE09C
:105A80002046FEF760FA05462B20065D95B1042DF1
:105A90000FD106F0200040B106F0040000B9E8E79D
:105AA00080212B200155002503E006F0040000B9F9
:105AB000052514E006F0040000B110E0A07900F024
:105AC000100008B905250AE0208AC0F3080207F192
:105AD00038001118384600F033F9A060C9E700BF5C
:105AE0002846BDE8FC81000010B5002821D0114BEC
:105AF0000022001F196803E0814203D80A46496862
:105B00000029F9D152B11368841A9C4204D100686B
:105B100018441060104602E0506000E0186039B18F
:105B200002680B1A934203D10B681A440260496859
:105B3000416010BD380000202DE9FF4F83B0804642
:105B400091461E460B224046049900F077F9052E37
:105B500018D9374611E039F802BB00250BE058464A
:105B600067F35F0007464FEA6B0B07F4803008B11C
:105B7000234847406D1C102DF1D3B9F800000028D0
:105B8000E9D13E46072500BF06F00F0000F1300ABC
:105B9000BAF1390F03DD0AF1070000F0FF0A2846C9
:105BA0006D1E01A901F800A03609002EECD17E205F
:105BB000485500240AE018F80400FEF725F920B142
:105BC000681EA04200D107E0641C641CAC4203D2F2
:105BD00018F804002028EED100BF00BF082D04D221
:105BE00028466D1C01A9085C00E020202146641CA9
:105BF00008F80100082CF1D307B0BDE8F08F0000D1
:105C0000211001002DE9F04781460C46D9F80050DB
:105C1000022C02D3E869A04202D84FF001085EE0EE
:105C20004FF0FF382878012804D002282CD0032810
:105C300051D13CE0264606EB5606A86A00EB5621F9
:105C4000284600F067FA00B148E03046761CC0F301
:105C5000080105F13800475CA86A00EB5621284688
:105C600000F058FA00B139E0C6F3080105F1380038
:105C7000405C47EA002704F0010008B1380901E060
:105C8000C7F30B00804629E0A86A00EB14212846E0
:105C900000F040FA00B121E040F2FF1101EA4402B5
:105CA00005F13801501800F06AF8804616E0A86A3D
:105CB00000EBD411284600F02DFA00B10EE040F2BE
:105CC000FF1101EA840205F13801501800F04BF889
:105CD00020F0704802E04FF0010800BF00BF4046CE
:105CE000BDE8F08700487047605B8F5470B504468C
:105CF0004FF0FF3026683146324601B970BD00BF13
:105D000012F8013B202B01D33A2BF9D13A2B11D1B8
:105D100001250E78302E08DB0E78392E05DC8E1C1E
:105D2000964202D10E78A6F13005012D01DA2846FF
:105D30002260E3E7014E307800BFDFE71A00002061
:105D400070B505460C4604F11A0000F018F8064636
:105D50002878032805D104F1140000F010F846EA71
:105D60000046304670BD0146C8788A7842EA002075
:105D70004A7842EA00200A7842EA00207047014649
:105D800048780A7842EA0020704710B50024FCF7F2
:105D9000ABFCFCF785FA044600BF002CFDDBFDF7E9
:105DA000F3FAFDF777FA002010BD0000F0B50B30D4
:105DB000154D20F007010024144A0FE003688B42C0
:105DC0000BD38B4205D95E1A43184768C3E90067B5
:105DD00000E04368136002C004E0021D1068002860
:105DE000ECD12046002802D1286808B10020F0BD7F
:105DF000064A07481060074A121A22F00702C0E953
:105E0000002401202860D7E73C0000203800002053
:105E10000404002000140020F0B503461D460C4683
:105E2000002000BF15F8017B14F801CBA7EB0C0094
:105E3000561E321E01D00028F4D0F0BD30B5034606
:105E40000C463AB100BF14F8015B03F8015B551E24
:105E50002A1EF8D130BD10B5034600BF03F8011B60
:105E6000541E221EFAD110BD2DE9F74F84B0002137
:105E7000059801600498FFF739FF03900398002804
:105E800003DA0B2007B0BDE8F08F9D49039851F865
:105E900020400CB90C20F5E705980460069800F046
:105EA000FE000690207878B16078FEF714FB074674
:105EB00007F0010040B9069820B107F0040008B1CE
:105EC0000A20DFE70020DDE70020207003986070E3
:105ED0006078FEF7A2FA074607F0010008B1032038
:105EE000D0E7069820B107F0040008B10A20C9E7FE
:105EF00000212046FFF756FD0546042D01D1012063
:105F0000C0E7022D01D30D20BCE7D4F8349004F192
:105F10004300FFF734FFB0F5007F01D00D20B1E75B
:105F200004F14E00FFF72BFF064626B904F15C0092
:105F3000FFF719FF064626624820005DA070A07892
:105F4000012804D0A078022801D00D209AE7A0787B
:105F500046434520005D6081608918B16089411E1B
:105F6000084008B10D208DE704F14900FFF707FF55
:105F70002081207A00F00F0008B10D2082E704F1A3
:105F80004B00FFF7FCFE8246BAF1000F04D104F18A
:105F90005800FFF7E8FE824604F14600FFF7EFFEE7
:105FA0008346BBF1000F01D10D206BE70BEB060020
:105FB000218900EB111002900298824501D20D2038
:105FC00060E70298AAEB00006189B0FBF1F8B8F134
:105FD000000F01D10D2055E700254A48804500D823
:105FE00003254FF6F570804500D8022540F6F57080
:105FF000804500D801250DB90D2043E708F10200C6
:10600000E061C4F8249009EB0B00A06202984844B8
:106010002063032D13D104F16200FFF7B0FE08B135
:106020000D202FE7208908B10D202BE704F1640033
:10603000FFF799FEE062E0698000019014E020899A
:1060400008B90D201EE7A06A3044E062022D02D19B
:10605000E069400007E0207F00F00100E16901EB0A
:10606000410100EB51000190216A019800F2FF10FC
:10607000B1EB502F01D20D2004E74FF0FF306061EB
:10608000206180202071032D2DD104F16800FFF7DD
:1060900076FE012827D109F10101204600F03AF8E7
:1060A00008BB0020207104F23620FFF768FE4AF694
:1060B0005521884217D104F13800FFF754FE1249E8
:1060C000884210D104F50770FFF74DFE0F49884252
:1060D00009D104F50870FFF746FE606104F5097008
:1060E000FFF741FE2061257009480088401C80B2FE
:1060F00007490880E0800020A06100BFC2E60000E0
:1061000014000020F5FFFF0F52526141727241618D
:106110001800002070B504460D460026606BA842AA
:1061200010D0204600F03EFA06465EB960780123A2
:106130002A4604F13801FEF7B3F910B14FF0FF35EC
:1061400001266563304670BD2DE9F04780460C4658
:1061500004F11A00FFF713FE10B10020BDE8F0872C
:10616000207820F04000401E00EB800101EBC005CC
:106170004FF00109002619E01549895D0819FFF75C
:10618000FEFD0746B9F1000F09D0FF2D01D900200F
:10619000E4E7B94628466D1C28F8107005E04FF674
:1061A000FF70874201D00020D8E7761C0D2EE3D384
:1061B000207800F0400048B1B9F1000F06D0FF2D63
:1061C00001D90020CAE7002028F815000120C5E702
:1061D000906600082DE9F04704460D4616464FF03C
:1061E0000209022D74D3E069A84271D920780128F0
:1061F00004D0022849D003280DD15EE02F4607EBDA
:106200005707A06A00EB57212046FFF783FF81461E
:10621000B9F1000F00D075E038467F1CC0F30801CB
:1062200004F1380001EB000805F0010028B1F1B2DB
:1062300098F8000061F31F1000E0304688F8000075
:106240000120E070A06A00EB57212046FFF762FFB3
:106250008146B9F1000F00D054E0C7F3080104F102
:10626000380001EB000805F0010010B1C6F307107B
:1062700006E098F8000000F0F000C6F303210843A0
:1062800088F800000120E0703CE0A06A00EB1521D6
:106290002046FFF73FFF8146B9F1000F00D031E003
:1062A000B1B240F2FF1202EA450304F13802981835
:1062B00000F019F90120E07024E0A06A00EBD5118C
:1062C0002046FFF727FF8146B9F1000F01D019E002
:1062D00019E040F2FF1101EA850204F1380150187B
:1062E000FFF741FD66F31B00064640F2FF1101EA8D
:1062F000850204F138015018314600F0E8F8012019
:10630000E07000BF00BF4846BDE8F0872DE9F047C8
:1063100007460C461546984684F80D800F20E0721B
:1063200000202073002104F11A0000F0DCF8681E40
:1063300000EB800101EBC00900200646824600BF49
:106340004FF6FF70864204D0484609F1010937F83C
:1063500010600D4911F80A100819314600F0C3F811
:106360000EB94FF6FF760AF1010082460D28E7D3F9
:106370004FF6FF70864202D037F8190008B945F091
:1063800040052570BDE8F08790660008F8B5044622
:106390000E4600BF6568002D00DAF8BDA7682846E4
:1063A0006D1C04F10C010E543C2D0CDB6B462A468F
:1063B0002068FFF765F90098A84201D1002001E0AC
:1063C0004FF0FF3005466560781CA06000BFE4E731
:1063D00038B50446606800280DDB6B4604F10C01FB
:1063E000D4E90002FFF74CF928B9606800998842A7
:1063F00001D1A06838BD4FF0FF30FBE770B504460F
:106400000D464C2200212046FFF725FD256070BD7A
:106410002DE9F04781460E4617464FF00008D9F89F
:106420000040022E02D3E069B04202D80220BDE84B
:10643000F08767B100BF4FF0FF3239462046FFF7C3
:10644000C9FE8046B8F1000F01D04046EFE700BF1B
:1064500031464846FFF7D6FB054605B922E0012D37
:1064600001D10220E3E7681C08B90120DFE7002220
:1064700031462046FFF7AEFE8046B8F1000F01D04E
:106480004046D4E7E069801E6169814206D26069B6
:10649000401C6061207940F0010020712E46E069C7
:1064A000B042D5D800BF0020C1E770B506460C4603
:1064B0001546A9B204F11A0000F015F83078032847
:1064C00004D1290C04F1140000F00DF870BD00F89F
:1064D000011B090A00F8011B090A00F8011B090A3F
:1064E00000F8011B704700F8011B091200F8011B9E
:1064F000704730B5014600200B2200BF431003EB6C
:10650000C01411F8015B6319D8B2531E1A1EF5D1DD
:1065100030BD000070B50446204600F043F8054643
:10652000002D38D1207803282ED1207901282BD1B5
:106530004202002104F13800FFF78DFC4AF6552194
:1065400004F23620FFF7CFFF144904F13800FFF7BB
:10655000BEFF134904F50770FFF7B9FF04F5087093
:106560006169FFF7B4FF04F509702169FFF7AFFF18
:10657000606A401C60636078012304F13801626B3B
:10658000FDF7AFFF00202071607800221146FDF773
:1065900057FF00B10125284670BD000052526141ED
:1065A0007272416170B504460025E078E8B1607808
:1065B000012304F13801626BFDF793FFA0B90020BD
:1065C000E070A16A606B401A216A88420DD2A078FF
:1065D00002280AD1236A616BCA186078012304F18A
:1065E0003801FDF77EFF00E00125284670BD2DE94A
:1065F000F0410646356815F8014B2046FDF704FCCE
:1066000060B115F8017B3846FDF704FC18B94FF06E
:10661000FF30BDE8F08107EB042084B24CB140F2BA
:10662000B5112046FFF730F9044614B94FF0FF309A
:10663000EFE7A04635604046EBE770B504460D46EF
:1066400009268CB1206878B12068007860B1A088F4
:106650002168C988884207D121684878FDF73BFF47
:1066600000F0010000B900260EB9206800E000200B
:106670002860304670BD00000000000000000102EC
:1066800003040607080900000000010203040000DB
:1066900001030507090E10121416181C1E809A45D6
:1066A000418E418F804545454949498E8F90929250
:1066B0004F994F555559999A9B9C9D9E9F41494F83
:1066C00055A5A5A6A7A8A9AAABACADAEAFB0B1B26F
:1066D000B3B4B5B6B7B8B9BABBBCBDBEBFC0C1C212
:1066E000C3C4C5C6C7C8C9CACBCCCDCECFD0D1D202
:1066F000D3D4D5D6D7D8D9DADBDCDDDEDFE0E1E2F2
:10670000E3E4E5E6E7E8E9EAEBECEDEEEFF0F1F2E1
:10671000F3F4F5F6F7F8F9FAFBFCFDFEFF000100D3
:10672000040010004000000100020000010002000F
:106730000400080010002000000000000700000016
:10674000000000000000000000000000C700FC0086
:10675000E900E200E400E000E500E700EA00EB0009
:10676000E800EF00EE00EC00C400C500C900E60040
:10677000C600F400F600F200FB00F900FF00D600AE
:10678000DC00A200A300A500A7209201E100ED001B
:10679000F300FA00F100D100AA00BA00BF001023F4
:1067A000AC00BD00BC00A100AB00BB009125922550
:1067B0009325022524256125622556255525632527
:1067C000512557255D255C255B251025142534258D
:1067D0002C251C2500253C255E255F255A255425A2
:1067E00069256625602550256C2567256825642563
:1067F000652559255825522553256B256A251825C9
:106800000C25882584258C2590258025B103DF0063
:106810009303C003A303C303B500C403A6039803F3
:10682000A903B4031E22C603B50329226122B100C5
:106830006522642220232123F7004822B000192278
:10684000B7001A227F20B200A025A00061001A0321
:10685000E0001703F8000703FF00010078010001C2
:10686000300132010601390110014A012E0179017E
:10687000060180014D0043028101820182018401F1
:10688000840186018701870189018A018B018B01BF
:106890008D018E018F01900191019101930194016D
:1068A000F60196019701980198013D029B019C0118
:1068B0009D0120029F01A001A001A201A201A4014B
:1068C000A401A601A701A701A901AA01AB01AC017E
:1068D000AC01AE01AF01AF01B101B201B301B3012F
:1068E000B501B501B701B801B801BA01BB01BC01DE
:1068F000BC01BE01F701C001C101C201C301C40155
:10690000C501C401C701C801C701CA01CB01CA0141
:10691000CD011001DD0101008E01DE011201F30144
:106920000300F101F401F401F8012801220212012F
:106930003A020900652C3B023B023D02662C3F02F5
:1069400040024102410246020A0153024000810115
:106950008601550289018A0158028F015A0290016D
:106960005C025D025E025F029301610262029401B9
:106970006402650266026702970196016A02622C50
:106980006C026D026E029C01700271029D01730225
:1069900074029F0176027702780279027A027B0202
:1069A0007C02642C7E027F02A60181028202A90180
:1069B0008402850286028702AE014402B101B2015F
:1069C00045028D028E028F0290029102B7017B0375
:1069D0000300FD03FE03FF03AC03040086038803EA
:1069E00089038A03B1031103C2030200A303A303B3
:1069F000C4030803CC0303008C038E038F03D80366
:106A00001801F2030A00F903F303F403F503F60394
:106A1000F703F703F903FA03FA03300420035004E1
:106A20001007600422018A043601C1040E01CF045C
:106A30000100C004D00444016105260400007D1D4E
:106A40000100632C001E9601A01E5A01001F0806BB
:106A5000101F0606201F0806301F0806401F0606E6
:106A6000511F0700591F521F5B1F541F5D1F561FE8
:106A70005F1F601F0806701F0E00BA1FBB1FC81FD4
:106A8000C91FCA1FCB1FDA1FDB1FF81FF91FEA1F20
:106A9000EB1FFA1FFB1F801F0806901F0806A01F90
:106AA0000806B01F0400B81FB91FB21FBC1FCC1FBF
:106AB0000100C31FD01F0206E01F0206E51F0100F0
:106AC000EC1FF31F0100FC1F4E2101003221702139
:106AD0001002842101008321D0241A05302C2F04B8
:106AE000602C0201672C0601752C0201802C6401C8
:106AF000002D260841FF1A0300002F5374617274A1
:106B000055702E696E690000404040404040404052
:106B10004041414141414040404040404040404070
:106B20004040404040404040050202020202020252
:106B30000202020202020202202020202020202045
:106B40002020020202020202029090909090901087
:106B50001010101010101010101010101010101035
:106B600010101002020202020288888888888808B1
:106B70000808080808080808080808080808080895
:106B80000808080202020240086B0008AC6B00080B
:106B9000000000204400000030350008F06B0008C1
:106BA00044000020BC150000403500080024F4001B
:106BB00000000000100000000100000000000000C4
:106BC00000000000000000537461727455700045AD
:106BD00078655061746800557064617465466C61D5
:106BE000670000000000000000000000000000003E
:0400000508000131BD
:00000001FF
